 unpack

 Timestamp is ffffffff (Sun Feb  7 06:28:15 2106)

 Preferred load address is 10000000

 Start         Length     Name                   Class
 0001:00000000 0000aa0eH .text$mn                CODE
 0002:00000000 000000ecH .idata$5                DATA
 0002:000000ec 00000004H .00cfg                  DATA
 0002:000000f0 00000004H .CRT$XCA                DATA
 0002:000000f4 00000004H .CRT$XCZ                DATA
 0002:000000f8 00000004H .CRT$XIA                DATA
 0002:000000fc 00000004H .CRT$XIZ                DATA
 0002:00000100 00000004H .CRT$XPA                DATA
 0002:00000104 00000004H .CRT$XPZ                DATA
 0002:00000108 00000004H .CRT$XTA                DATA
 0002:0000010c 00000004H .CRT$XTZ                DATA
 0002:00000110 00000000H .gfids$y                DATA
 0002:00000110 00002620H .rdata                  DATA
 0002:00002730 00000130H .rdata$r                DATA
 0002:00002860 00000004H .rdata$sxdata           DATA
 0002:00002864 000002a8H .rdata$zzzdbg           DATA
 0002:00002b0c 00000004H .rtc$IAA                DATA
 0002:00002b10 00000004H .rtc$IZZ                DATA
 0002:00002b14 00000004H .rtc$TAA                DATA
 0002:00002b18 00000008H .rtc$TZZ                DATA
 0002:00002b20 00000110H .xdata$x                DATA
 0002:00002c30 00000214H .edata                  DATA
 0002:00002e44 000000dcH .idata$2                DATA
 0002:00002f20 00000014H .idata$3                DATA
 0002:00002f34 000000ecH .idata$4                DATA
 0002:00003020 0000048aH .idata$6                DATA
 0003:00000000 00000b18H .data                   DATA
 0003:00000b18 00000078H .data$r                 DATA
 0003:00000b90 0000078cH .bss                    DATA
 0004:00000000 00000060H .rsrc$01                DATA
 0004:00000060 00000310H .rsrc$02                DATA

  Address         Publics by Value              Rva+Base       Lib:Object

 0000:00000000       ___guard_fids_table        00000000     <absolute>
 0000:00000000       ___guard_iat_table         00000000     <absolute>
 0000:00000000       ___dynamic_value_reloc_table 00000000     <absolute>
 0000:00000000       ___hybrid_code_map         00000000     <absolute>
 0000:00000000       ___guard_fids_count        00000000     <absolute>
 0000:00000000       ___guard_iat_count         00000000     <absolute>
 0000:00000000       ___hybrid_auxiliary_iat    00000000     <absolute>
 0000:00000000       ___enclave_config          00000000     <absolute>
 0000:00000000       ___guard_longjmp_count     00000000     <absolute>
 0000:00000000       ___volatile_metadata       00000000     <absolute>
 0000:00000000       ___hybrid_code_map_count   00000000     <absolute>
 0000:00000000       ___guard_longjmp_table     00000000     <absolute>
 0000:00000001       ___safe_se_handler_count   00000001     <absolute>
 0000:00000100       ___guard_flags             00000100     <absolute>
 0000:00000000       ___ImageBase               10000000     <linker-defined>
 0001:00000000       ?getIndex@cpool@@QAEPAUcpindex@@C@Z 10001000 f i bands.obj
 0001:0000001d       ?getIntCount@band@@QAEHH@Z 1000101d f   bands.obj
 0001:000000ea       ?getIntTotal@band@@QAEHXZ  100010ea f   bands.obj
 0001:00000161       ?getLong@band@@QAE_JAAU1@_N@Z 10001161 f   bands.obj
 0001:00000196       ?getRefCommon@band@@QAEPAUentry@@PAUcpindex@@_N@Z 10001196 f   bands.obj
 0001:00000207       ?initIndexes@band@@SAXPAUunpacker@@@Z 10001207 f   bands.obj
 0001:0000024c       ?makeBands@band@@SAPAU1@PAUunpacker@@@Z 1000124c f   bands.obj
 0001:000002d0       ?readData@band@@QAEXH@Z    100012d0 f   bands.obj
 0001:00000480       ?setIndex@band@@QAEXPAUcpindex@@@Z 10001480 f   bands.obj
 0001:0000048a       ?setIndexByTag@band@@QAEXC@Z 1000148a f   bands.obj
 0001:000004a6       ?compareTo@bytes@@QAEHAAU1@@Z 100014a6 f   bytes.obj
 0001:000004dd       ?copyFrom@bytes@@QAEXPBXII@Z 100014dd f   bytes.obj
 0001:000004f7       ?ensureSize@fillbytes@@QAEXI@Z 100014f7 f   bytes.obj
 0001:00000517       ?free@bytes@@QAEXXZ        10001517 f   bytes.obj
 0001:00000539       ?freeAll@ptrlist@@QAEXXZ   10001539 f   bytes.obj
 0001:00000576       ?grow@fillbytes@@QAEPACI@Z 10001576 f   bytes.obj
 0001:0000060d       ?indexOf@ptrlist@@QAEHPBX@Z 1000160d f   bytes.obj
 0001:00000633       ?malloc@bytes@@QAEXI@Z     10001633 f   bytes.obj
 0001:00000682       ?realloc@bytes@@QAEXI@Z    10001682 f   bytes.obj
 0001:00000718       ?saveFrom@bytes@@QAEXPBXI@Z 10001718 f   bytes.obj
 0001:00000740       ?writeTo@bytes@@QAEPACPAC@Z 10001740 f   bytes.obj
 0001:00000787       ?findByIndex@coding@@SAPAU1@H@Z 10001787 f   coding.obj
 0001:000007a4       ?findBySpec@coding@@SAPAU1@H@Z 100017a4 f   coding.obj
 0001:000007ff       ?findBySpec@coding@@SAPAU1@HHHH@Z 100017ff f   coding.obj
 0001:00000844       ?free@coding@@QAEXXZ       10001844 f   coding.obj
 0001:0000087b       ?getInt@value_stream@@QAEHXZ 1000187b f   coding.obj
 0001:00000aea       ?init@coding@@QAEPAU1@XZ   10001aea f   coding.obj
 0001:00000d37       ?init@coding_method@@QAEXAAPACPAC0HPAUcoding@@HPAUintlist@@@Z 10001d37 f   coding.obj
 0001:000013da       ?init@value_stream@@QAEXPAC0PAUcoding@@@Z 100023da f   coding.obj
 0001:000013fc       ?parse@coding@@SAIAAPACHH@Z 100023fc f   coding.obj
 0001:00001460       ?parseMultiple@coding@@SAXAAPACHPACHH@Z 10002460 f   coding.obj
 0001:000014eb       ?parse_lgH@coding@@SAIAAPACHHH@Z 100024eb f   coding.obj
 0001:0000154c       ?reset@coding_method@@QAEXPAUvalue_stream@@@Z 1000254c f   coding.obj
 0001:0000156e       ?setCoding@value_stream@@QAEXPAUcoding@@@Z 1000256e f   coding.obj
 0001:0000166e       ?sumInUnsignedRange@coding@@QAEHHH@Z 1000266e f   coding.obj
 0001:0000169a       ?CallLongMethod@JNIEnv_@@QAA_JPAV_jobject@@PAU_jmethodID@@ZZ 1000269a f i jni.obj
 0001:000016b5       ?CallStaticObjectMethod@JNIEnv_@@QAAPAV_jobject@@PAV_jclass@@PAU_jmethodID@@ZZ 100026b5 f i jni.obj
 0001:000016d0       ?SetLongField@JNIEnv_@@QAEXPAV_jobject@@PAU_jfieldID@@_J@Z 100026d0 f i jni.obj
 0001:000016ec       ?current@unpacker@@SAPAU1@XZ 100026ec f   jni.obj
 0001:0000188d       _Java_com_sun_java_util_jar_pack_NativeUnpack_finish@8 1000288d f   jni.obj
 0001:000018d8       _Java_com_sun_java_util_jar_pack_NativeUnpack_getNextFile@12 100028d8 f   jni.obj
 0001:00001a6e       _Java_com_sun_java_util_jar_pack_NativeUnpack_getOption@12 10002a6e f   jni.obj
 0001:00001aed       _Java_com_sun_java_util_jar_pack_NativeUnpack_getUnusedInput@8 10002aed f   jni.obj
 0001:00001b75       _Java_com_sun_java_util_jar_pack_NativeUnpack_initIDs@8 10002b75 f   jni.obj
 0001:00001c4f       _Java_com_sun_java_util_jar_pack_NativeUnpack_setOption@16 10002c4f f   jni.obj
 0001:00001ce7       _Java_com_sun_java_util_jar_pack_NativeUnpack_start@20 10002ce7 f   jni.obj
 0001:00001da9       ?abort@unpacker@@QAEXPBD@Z 10002da9 f   unpack.obj
 0001:00001dee       ?add_size@@YAIIIH@Z        10002dee f i unpack.obj
 0001:00001e25       ?buildBands@attr_definitions@unpacker@@QAEPAPAUband@@PAUlayout_definition@2@@Z 10002e25 f   unpack.obj
 0001:00001f4a       ?calloc_heap@unpacker@@QAEPAXII_N0@Z 10002f4a f   unpack.obj
 0001:00002002       ?checkLegacy@unpacker@@QAEXPBD@Z 10003002 f   unpack.obj
 0001:00002055       ?check_options@unpacker@@QAEXXZ 10003055 f   unpack.obj
 0001:00002092       ?close_output@unpacker@@QAEPAUfillbytes@@PAU2@@Z 10003092 f   unpack.obj
 0001:00002175       ?computeOutputIndexes@cpool@@QAEXXZ 10003175 f   unpack.obj
 0001:000021cd       ?defineLayout@attr_definitions@unpacker@@QAEPAUlayout_definition@2@HPAUentry@@PBD@Z 100031cd f i unpack.obj
 0001:000021f9       ?defineLayout@attr_definitions@unpacker@@QAEPAUlayout_definition@2@HPBD0@Z 100031f9 f   unpack.obj
 0001:000022e2       ?ensureClass@cpool@@QAEPAUentry@@AAUbytes@@@Z 100032e2 f   unpack.obj
 0001:0000237a       ?ensureUtf8@cpool@@QAEPAUentry@@AAUbytes@@@Z 1000337a f   unpack.obj
 0001:000023f4       ?ensure_input@unpacker@@QAE_N_J@Z 100033f4 f   unpack.obj
 0001:0000254f       ?ensure_put_space@unpacker@@QAEXI@Z 1000354f f   unpack.obj
 0001:00002597       ?expandSignatures@cpool@@QAEXXZ 10003597 f   unpack.obj
 0001:00002746       ?free@attr_definitions@unpacker@@QAEXXZ 10003746 f i unpack.obj
 0001:000027b9       ?free@jar@@QAEXXZ          100037b9 f i unpack.obj
 0001:000027e4       ?free@unpacker@@QAEXXZ     100037e4 f   unpack.obj
 0001:00002989       ?free_temps@unpacker@@QAEXXZ 10003989 f i unpack.obj
 0001:0000299c       ?get@cpindex@@QAEPAUentry@@I@Z 1000399c f   unpack.obj
 0001:000029c1       ?getCount@attr_definitions@unpacker@@QAEAAHI@Z 100039c1 f i unpack.obj
 0001:000029e1       ?getFieldIndex@cpool@@QAEPAUcpindex@@PAUentry@@@Z 100039e1 f i unpack.obj
 0001:00002a0c       ?getFirstChildIC@cpool@@QAEPAUinner_class@@PAUentry@@@Z 10003a0c f   unpack.obj
 0001:00002a2c       ?getIC@cpool@@QAEPAUinner_class@@PAUentry@@@Z 10003a2c f   unpack.obj
 0001:00002a4c       ?getKQIndex@cpool@@QAEPAUcpindex@@XZ 10003a4c f   unpack.obj
 0001:00002acf       ?getLayout@attr_definitions@unpacker@@QAEPAUlayout_definition@2@I@Z 10003acf f i unpack.obj
 0001:00002aea       ?getMethodIndex@cpool@@QAEPAUcpindex@@PAUentry@@@Z 10003aea f i unpack.obj
 0001:00002b1c       ?get_abort_message@unpacker@@QAEPBDXZ 10003b1c f   unpack.obj
 0001:00002b20       ?get_code_header@unpacker@@QAEXAAH000@Z 10003b20 f   unpack.obj
 0001:00002bbd       ?get_next_file@unpacker@@QAEPAUfile@1@XZ 10003bbd f   unpack.obj
 0001:00002f1c       ?get_option@unpacker@@QAEPBDPBD@Z 10003f1c f   unpack.obj
 0001:00002fd0       ?hashTabRef@cpool@@QAEAAPAUentry@@CAAUbytes@@@Z 10003fd0 f   unpack.obj
 0001:0000308c       ?init@band@@QAEXPAUunpacker@@HH@Z 1000408c f i unpack.obj
 0001:000030b4       ?init@cpool@@QAEXPAUunpacker@@QAH@Z 100040b4 f   unpack.obj
 0001:00003235       ?init@unpacker@@QAEXP6A_JPAU1@PAX_J2@Z@Z 10004235 f   unpack.obj
 0001:000032ab       ?initGroupIndexes@cpool@@QAEXXZ 100042ab f   unpack.obj
 0001:00003372       ?initMemberIndexes@cpool@@QAEXXZ 10004372 f   unpack.obj
 0001:000035d5       ?isIndex@attr_definitions@unpacker@@QAE_NI@Z 100045d5 f i unpack.obj
 0001:00003627       ?isPredefined@attr_definitions@unpacker@@QAE_NI@Z 10004627 f i unpack.obj
 0001:00003652       ?isRedefined@attr_definitions@unpacker@@QAE_NI@Z 10004652 f i unpack.obj
 0001:000036e7       ?parseIntLayout@attr_definitions@unpacker@@QAEPBDPBDAAPAUband@@C_N@Z 100046e7 f   unpack.obj
 0001:000037bb       ?parseLayout@attr_definitions@unpacker@@QAEPBDPBDAAPAPAUband@@H@Z 100047bb f   unpack.obj
 0001:00003ebf       ?parseNumeral@attr_definitions@unpacker@@QAEPBDPBDAAH@Z 10004ebf f   unpack.obj
 0001:00003f58       ?popBody@attr_definitions@unpacker@@QAEPAPAUband@@H@Z 10004f58 f   unpack.obj
 0001:00003fd6       ?predefCount@attr_definitions@unpacker@@QAEHI@Z 10004fd6 f   unpack.obj
 0001:00003ff5       ?put_bytes@unpacker@@QAEXAAUbytes@@@Z 10004ff5 f i unpack.obj
 0001:0000400e       ?put_label@unpacker@@QAEXHH@Z 1000500e f   unpack.obj
 0001:0000405c       ?put_space@unpacker@@QAEPACI@Z 1000505c f   unpack.obj
 0001:00004091       ?put_stackmap_type@unpacker@@QAEXXZ 10005091 f   unpack.obj
 0001:00004104       ?putlayout@unpacker@@QAEXPAPAUband@@@Z 10005104 f   unpack.obj
 0001:0000430f       ?putref@unpacker@@QAEXPAUentry@@@Z 1000530f f   unpack.obj
 0001:00004333       ?putref_index@unpacker@@QAEHPAUentry@@H@Z 10005333 f   unpack.obj
 0001:000043b7       ?putu1ref@unpacker@@QAEXPAUentry@@@Z 100053b7 f   unpack.obj
 0001:000043d8       ?putu2@unpacker@@QAEXH@Z   100053d8 f   unpack.obj
 0001:000043ee       ?putu2_at@unpacker@@SAXPACH@Z 100053ee f   unpack.obj
 0001:00004417       ?putu4@unpacker@@QAEXH@Z   10005417 f   unpack.obj
 0001:0000442d       ?putu4_at@unpacker@@SAXPACH@Z 1000542d f   unpack.obj
 0001:00004450       ?putu8@unpacker@@QAEX_J@Z  10005450 f   unpack.obj
 0001:0000446b       ?putu8_at@unpacker@@SAXPAC_J@Z 1000546b f   unpack.obj
 0001:0000448c       ?readBandData@attr_definitions@unpacker@@QAEXH@Z 1000548c f   unpack.obj
 0001:00004520       ?readBandData@attr_definitions@unpacker@@QAEXPAPAUband@@I@Z 10005520 f   unpack.obj
 0001:00004659       ?read_Utf8_values@unpacker@@QAEXPAUentry@@HC@Z 10005659 f i unpack.obj
 0001:00004c24       ?read_attr_defs@unpacker@@QAEXXZ 10005c24 f   unpack.obj
 0001:00004edb       ?read_attrs@unpacker@@QAEXHH@Z 10005edb f   unpack.obj
 0001:00005876       ?read_bands@unpacker@@QAEXXZ 10006876 f   unpack.obj
 0001:000058e2       ?read_bcs@unpacker@@QAEXXZ 100068e2 f i unpack.obj
 0001:00005c47       ?read_bootstrap_methods@unpacker@@QAEXPAUentry@@HC@Z 10006c47 f   unpack.obj
 0001:00005d84       ?read_classes@unpacker@@QAEXXZ 10006d84 f   unpack.obj
 0001:00005eb2       ?read_code_headers@unpacker@@QAEXXZ 10006eb2 f   unpack.obj
 0001:0000601b       ?read_cp@unpacker@@QAEXXZ  1000701b f   unpack.obj
 0001:000062ef       ?read_double_refs@unpacker@@QAEXAAUband@@CCPAUentry@@HC@Z 100072ef f   unpack.obj
 0001:000063b9       ?read_double_words@unpacker@@QAEXAAUband@@PAUentry@@HCH@Z 100073b9 f   unpack.obj
 0001:0000644a       ?read_file_header@unpacker@@QAEXXZ 1000744a f   unpack.obj
 0001:00006ba0       ?read_files@unpacker@@QAEXXZ 10007ba0 f   unpack.obj
 0001:00006c9b       ?read_ics@unpacker@@QAEXXZ 10007c9b f   unpack.obj
 0001:0000700e       ?read_method_handle@unpacker@@QAEXPAUentry@@HCH@Z 1000800e f   unpack.obj
 0001:00007103       ?read_method_type@unpacker@@QAEXPAUentry@@HCH@Z 10008103 f   unpack.obj
 0001:000071ce       ?read_signature_values@unpacker@@QAEXPAUentry@@HC@Z 100081ce f   unpack.obj
 0001:0000734f       ?read_single_refs@unpacker@@QAEXAAUband@@CPAUentry@@HCH@Z 1000834f f   unpack.obj
 0001:00007453       ?read_single_words@unpacker@@QAEXAAUband@@PAUentry@@HCH@Z 10008453 f i unpack.obj
 0001:000074cd       ?redirect_stdio@unpacker@@QAEXXZ 100084cd f   unpack.obj
 0001:00007565       ?ref_band_for_op@unpacker@@QAEPAUband@@H@Z 10008565 f   unpack.obj
 0001:000076a1       ?ref_band_for_self_op@unpacker@@QAEPAUband@@HAA_NAAH@Z 100086a1 f   unpack.obj
 0001:00007718       ?requestOutputIndex@entry@@QAEXAAUcpool@@H@Z 10008718 f   unpack.obj
 0001:00007789       ?resetOutputIndexes@cpool@@QAEXXZ 10008789 f   unpack.obj
 0001:000077de       ?reset_cur_classfile@unpacker@@QAEXXZ 100087de f   unpack.obj
 0001:00007826       ?saveIntStr@unpacker@@QAEPBDH@Z 10008826 f i unpack.obj
 0001:00007867       ?saveStr@unpacker@@QAEPBDPBD@Z 10008867 f i unpack.obj
 0001:0000788f       ?saveTo@unpacker@@QAEXAAUbytes@@PACI@Z 1000888f f   unpack.obj
 0001:000078e1       ?scale_size@@YAIII@Z       100088e1 f i unpack.obj
 0001:00007902       ?set_option@unpacker@@QAE_NPBD0@Z 10008902 f   unpack.obj
 0001:00007a51       ?set_output@unpacker@@QAEXPAUfillbytes@@@Z 10008a51 f i unpack.obj
 0001:00007a88       ?start@unpacker@@QAEXPAXI@Z 10008a88 f   unpack.obj
 0001:00007b11       ?to_bci@unpacker@@QAEII@Z  10008b11 f   unpack.obj
 0001:00007b62       ?typeSize@entry@@QAEHXZ    10008b62 f   unpack.obj
 0001:00007bd8       ?utf8String@entry@@QAEPBDXZ 10008bd8 f i unpack.obj
 0001:00007bfc       ?write_attrs@unpacker@@QAEHH_K@Z 10008bfc f   unpack.obj
 0001:00008684       ?write_bc_ops@unpacker@@QAEXXZ 10009684 f i unpack.obj
 0001:00008e53       ?write_bsms@unpacker@@QAEHHH@Z 10009e53 f   unpack.obj
 0001:00008f5d       ?write_classfile_head@unpacker@@QAEXXZ 10009f5d f   unpack.obj
 0001:000090b7       ?write_classfile_tail@unpacker@@QAEXXZ 1000a0b7 f   unpack.obj
 0001:000092ec       ?write_code@unpacker@@QAEXXZ 1000a2ec f i unpack.obj
 0001:000094c3       ?write_ics@unpacker@@QAEHHH@Z 1000a4c3 f   unpack.obj
 0001:0000981e       ?write_members@unpacker@@QAEXHH@Z 1000a81e f   unpack.obj
 0001:00009958       ___local_stdio_printf_options 1000a958 f i unpack.obj
 0001:0000995e       __snprintf                 1000a95e f i unpack.obj
 0001:00009978       __vfprintf_l               1000a978 f i unpack.obj
 0001:0000999c       __vsnprintf                1000a99c f i unpack.obj
 0001:000099b7       __vsnprintf_l              1000a9b7 f i unpack.obj
 0001:000099ea       _fprintf                   1000a9ea f i unpack.obj
 0001:00009a02       _outputEntry_cmp           1000aa02 f   unpack.obj
 0001:00009a73       _raw_address_cmp           1000aa73 f   unpack.obj
 0001:00009a8e       _sprintf                   1000aa8e f i unpack.obj
 0001:00009aa8       ?must_calloc@@YAPAXII@Z    1000aaa8 f   utils.obj
 0001:00009aeb       ?unpack_abort@@YAXPBDPAUunpacker@@@Z 1000aaeb f   utils.obj
 0001:00009b34       ?unpack_aborting@@YA_NPAUunpacker@@@Z 1000ab34 f   utils.obj
 0001:00009b69       ?free@gunzip@@QAEXXZ       1000ab69 f   zip.obj
 0001:00009b69       @_guard_check_icall_nop@4  1000ab69 f   MSVCRT:guard_support.obj
 0001:00009b6a       ?init@jar@@QAEXPAUunpacker@@@Z 1000ab6a f   zip.obj
 0001:00009b88       _JNU_ThrowIOException@8    1000ab88 f   java:java.dll
 0001:00009b8e       @__security_check_cookie@4 1000ab8e f   MSVCRT:secchk.obj
 0001:00009ba0       __allmul                   1000aba0 f   MSVCRT:llmul.obj
 0001:00009bd4       ??2@YAPAXI@Z               1000abd4 f   MSVCRT:new_scalar.obj
 0001:00009c04       ??3@YAXPAXI@Z              1000ac04 f   MSVCRT:delete_scalar_size.obj
 0001:00009c20       __aullshr                  1000ac20 f   MSVCRT:ullshr.obj
 0001:00009f5f       __DllMainCRTStartup@12     1000af5f f   MSVCRT:dll_dllmain.obj
 0001:00009f82       ___raise_securityfailure   1000af82 f   MSVCRT:gs_report.obj
 0001:00009fac       ___report_gsfailure        1000afac f   MSVCRT:gs_report.obj
 0001:0000a0a5       ??0bad_alloc@std@@QAE@ABV01@@Z 1000b0a5 f i MSVCRT:throw_bad_alloc.obj
 0001:0000a0c0       ??0bad_alloc@std@@QAE@XZ   1000b0c0 f i MSVCRT:throw_bad_alloc.obj
 0001:0000a0d8       ??0bad_array_new_length@std@@QAE@ABV01@@Z 1000b0d8 f i MSVCRT:throw_bad_alloc.obj
 0001:0000a0f3       ??0bad_array_new_length@std@@QAE@XZ 1000b0f3 f i MSVCRT:throw_bad_alloc.obj
 0001:0000a10b       ??0exception@std@@QAE@ABV01@@Z 1000b10b f i MSVCRT:throw_bad_alloc.obj
 0001:0000a137       ??1bad_alloc@std@@UAE@XZ   1000b137 f i MSVCRT:throw_bad_alloc.obj
 0001:0000a137       ??1bad_array_new_length@std@@UAE@XZ 1000b137 f i MSVCRT:throw_bad_alloc.obj
 0001:0000a148       ??_Gbad_array_new_length@std@@UAEPAXI@Z 1000b148 f i MSVCRT:throw_bad_alloc.obj
 0001:0000a148       ??_Ebad_alloc@std@@UAEPAXI@Z 1000b148 f i MSVCRT:throw_bad_alloc.obj
 0001:0000a148       ??_Ebad_array_new_length@std@@UAEPAXI@Z 1000b148 f i MSVCRT:throw_bad_alloc.obj
 0001:0000a148       ??_Eexception@std@@UAEPAXI@Z 1000b148 f i MSVCRT:throw_bad_alloc.obj
 0001:0000a148       ??_Gbad_alloc@std@@UAEPAXI@Z 1000b148 f i MSVCRT:throw_bad_alloc.obj
 0001:0000a148       ??_Gexception@std@@UAEPAXI@Z 1000b148 f i MSVCRT:throw_bad_alloc.obj
 0001:0000a175       ?__scrt_throw_std_bad_alloc@@YAXXZ 1000b175 f   MSVCRT:throw_bad_alloc.obj
 0001:0000a192       ?__scrt_throw_std_bad_array_new_length@@YAXXZ 1000b192 f   MSVCRT:throw_bad_alloc.obj
 0001:0000a1af       ?what@exception@std@@UBEPBDXZ 1000b1af f i MSVCRT:throw_bad_alloc.obj
 0001:0000a1bc       ??3@YAXPAX@Z               1000b1bc f   MSVCRT:delete_scalar.obj
 0001:0000a20e       ___security_init_cookie    1000b20e f   MSVCRT:gs_support.obj
 0001:0000a259       _DllMain@12                1000b259 f   MSVCRT:dll_dllmain_stub.obj
 0001:0000a27b       ?__scrt_initialize_type_info@@YAXXZ 1000b27b f   MSVCRT:tncleanup.obj
 0001:0000a287       ?__scrt_uninitialize_type_info@@YAXXZ 1000b287 f   MSVCRT:tncleanup.obj
 0001:0000a293       ___local_stdio_scanf_options 1000b293 f i MSVCRT:default_local_stdio_options.obj
 0001:0000a299       ___scrt_initialize_default_local_stdio_options 1000b299 f   MSVCRT:default_local_stdio_options.obj
 0001:0000a2fa       ___scrt_acquire_startup_lock 1000b2fa f   MSVCRT:utility.obj
 0001:0000a32c       ___scrt_dllmain_after_initialize_c 1000b32c f   MSVCRT:utility.obj
 0001:0000a357       ___scrt_dllmain_before_initialize_c 1000b357 f   MSVCRT:utility.obj
 0001:0000a365       ___scrt_dllmain_crt_thread_attach 1000b365 f   MSVCRT:utility.obj
 0001:0000a384       ___scrt_dllmain_crt_thread_detach 1000b384 f   MSVCRT:utility.obj
 0001:0000a391       ___scrt_dllmain_exception_filter 1000b391 f   MSVCRT:utility.obj
 0001:0000a3c5       ___scrt_dllmain_uninitialize_c 1000b3c5 f   MSVCRT:utility.obj
 0001:0000a3e8       ___scrt_dllmain_uninitialize_critical 1000b3e8 f   MSVCRT:utility.obj
 0001:0000a3f5       ___scrt_initialize_crt     1000b3f5 f   MSVCRT:utility.obj
 0001:0000a42e       ___scrt_initialize_onexit_tables 1000b42e f   MSVCRT:utility.obj
 0001:0000a4d3       ___scrt_is_nonwritable_in_current_image 1000b4d3 f   MSVCRT:utility.obj
 0001:0000a567       ___scrt_release_startup_lock 1000b567 f   MSVCRT:utility.obj
 0001:0000a584       ___scrt_uninitialize_crt   1000b584 f   MSVCRT:utility.obj
 0001:0000a5ac       ___scrt_get_dyn_tls_init_callback 1000b5ac f   MSVCRT:dyn_tls_init.obj
 0001:0000a5b2       ___scrt_fastfail           1000b5b2 f   MSVCRT:utility_desktop.obj
 0001:0000a6cc       __crt_debugger_hook        1000b6cc f   MSVCRT:utility_desktop.obj
 0001:0000a6d4       __RTC_Initialize           1000b6d4 f   MSVCRT:initsect.obj
 0001:0000a700       __RTC_Terminate            1000b700 f   MSVCRT:initsect.obj
 0001:0000a730       __SEH_prolog4              1000b730 f   MSVCRT:sehprolg4.obj
 0001:0000a776       __SEH_epilog4              1000b776 f   MSVCRT:sehprolg4.obj
 0001:0000a78b       __except_handler4          1000b78b f   MSVCRT:chandler4gs.obj
 0001:0000a7ae       ??_Etype_info@@UAEPAXI@Z   1000b7ae f i MSVCRT:std_type_info_static.obj
 0001:0000a7ae       ??_Gtype_info@@UAEPAXI@Z   1000b7ae f i MSVCRT:std_type_info_static.obj
 0001:0000a7d1       ___isa_available_init      1000b7d1 f   MSVCRT:cpu_disp.obj
 0001:0000a968       __get_startup_argv_mode    1000b968 f   MSVCRT:argv_mode.obj
 0001:0000a96c       ___scrt_is_ucrt_dll_in_use 1000b96c f   MSVCRT:ucrt_detection.obj
 0001:0000a978       _IsProcessorFeaturePresent@4 1000b978 f   kernel32:KERNEL32.dll
 0001:0000a97e       _memcmp                    1000b97e f   vcruntime:VCRUNTIME140.dll
 0001:0000a984       _memcpy                    1000b984 f   vcruntime:VCRUNTIME140.dll
 0001:0000a98a       _memset                    1000b98a f   vcruntime:VCRUNTIME140.dll
 0001:0000a990       _strchr                    1000b990 f   vcruntime:VCRUNTIME140.dll
 0001:0000a996       ___std_exception_copy      1000b996 f   vcruntime:VCRUNTIME140.dll
 0001:0000a99c       ___std_exception_destroy   1000b99c f   vcruntime:VCRUNTIME140.dll
 0001:0000a9a2       __CxxThrowException@8      1000b9a2 f   vcruntime:VCRUNTIME140.dll
 0001:0000a9a8       ___std_type_info_destroy_list 1000b9a8 f   vcruntime:VCRUNTIME140.dll
 0001:0000a9ae       __except_handler4_common   1000b9ae f   vcruntime:VCRUNTIME140.dll
 0001:0000a9b4       _free                      1000b9b4 f   ucrt:api-ms-win-crt-heap-l1-1-0.dll
 0001:0000a9ba       _strcat                    1000b9ba f   ucrt:api-ms-win-crt-string-l1-1-0.dll
 0001:0000a9c0       _strcmp                    1000b9c0 f   ucrt:api-ms-win-crt-string-l1-1-0.dll
 0001:0000a9c6       _strlen                    1000b9c6 f   ucrt:api-ms-win-crt-string-l1-1-0.dll
 0001:0000a9cc       __callnewh                 1000b9cc f   ucrt:api-ms-win-crt-heap-l1-1-0.dll
 0001:0000a9d2       _malloc                    1000b9d2 f   ucrt:api-ms-win-crt-heap-l1-1-0.dll
 0001:0000a9d8       __initterm                 1000b9d8 f   ucrt:api-ms-win-crt-runtime-l1-1-0.dll
 0001:0000a9de       __initterm_e               1000b9de f   ucrt:api-ms-win-crt-runtime-l1-1-0.dll
 0001:0000a9e4       __seh_filter_dll           1000b9e4 f   ucrt:api-ms-win-crt-runtime-l1-1-0.dll
 0001:0000a9ea       __configure_narrow_argv    1000b9ea f   ucrt:api-ms-win-crt-runtime-l1-1-0.dll
 0001:0000a9f0       __initialize_narrow_environment 1000b9f0 f   ucrt:api-ms-win-crt-runtime-l1-1-0.dll
 0001:0000a9f6       __initialize_onexit_table  1000b9f6 f   ucrt:api-ms-win-crt-runtime-l1-1-0.dll
 0001:0000a9fc       __execute_onexit_table     1000b9fc f   ucrt:api-ms-win-crt-runtime-l1-1-0.dll
 0001:0000aa02       __cexit                    1000ba02 f   ucrt:api-ms-win-crt-runtime-l1-1-0.dll
 0001:0000aa08       ___acrt_thread_detach      1000ba08 f   MSVCRT:ucrt_stubs.obj
 0001:0000aa08       ___scrt_stub_for_acrt_uninitialize_critical 1000ba08 f   MSVCRT:ucrt_stubs.obj
 0001:0000aa08       ___vcrt_thread_attach      1000ba08 f   MSVCRT:ucrt_stubs.obj
 0001:0000aa08       ___vcrt_thread_detach      1000ba08 f   MSVCRT:ucrt_stubs.obj
 0001:0000aa08       ___acrt_thread_attach      1000ba08 f   MSVCRT:ucrt_stubs.obj
 0001:0000aa08       ___scrt_stub_for_acrt_initialize 1000ba08 f   MSVCRT:ucrt_stubs.obj
 0001:0000aa08       ___acrt_initialize         1000ba08 f   MSVCRT:ucrt_stubs.obj
 0001:0000aa08       ___scrt_stub_for_acrt_thread_attach 1000ba08 f   MSVCRT:ucrt_stubs.obj
 0001:0000aa08       ___acrt_uninitialize       1000ba08 f   MSVCRT:ucrt_stubs.obj
 0001:0000aa08       ___vcrt_uninitialize       1000ba08 f   MSVCRT:ucrt_stubs.obj
 0001:0000aa08       ___acrt_uninitialize_critical 1000ba08 f   MSVCRT:ucrt_stubs.obj
 0001:0000aa08       ___vcrt_uninitialize_critical 1000ba08 f   MSVCRT:ucrt_stubs.obj
 0001:0000aa08       ___scrt_stub_for_acrt_thread_detach 1000ba08 f   MSVCRT:ucrt_stubs.obj
 0001:0000aa08       ___scrt_stub_for_acrt_uninitialize 1000ba08 f   MSVCRT:ucrt_stubs.obj
 0001:0000aa08       ___vcrt_initialize         1000ba08 f   MSVCRT:ucrt_stubs.obj
 0001:0000aa0b       __is_c_termination_complete 1000ba0b f   MSVCRT:ucrt_stubs.obj
 0001:0000aa0b       ___scrt_stub_for_is_c_termination_complete 1000ba0b f   MSVCRT:ucrt_stubs.obj
 0002:00000000       __imp__IsDebuggerPresent@0 1000c000     kernel32:KERNEL32.dll
 0002:00000004       __imp__InitializeSListHead@4 1000c004     kernel32:KERNEL32.dll
 0002:00000008       __imp__UnhandledExceptionFilter@4 1000c008     kernel32:KERNEL32.dll
 0002:0000000c       __imp__SetUnhandledExceptionFilter@4 1000c00c     kernel32:KERNEL32.dll
 0002:00000010       __imp__GetCurrentProcess@0 1000c010     kernel32:KERNEL32.dll
 0002:00000014       __imp__TerminateProcess@8  1000c014     kernel32:KERNEL32.dll
 0002:00000018       __imp__IsProcessorFeaturePresent@4 1000c018     kernel32:KERNEL32.dll
 0002:0000001c       __imp__QueryPerformanceCounter@4 1000c01c     kernel32:KERNEL32.dll
 0002:00000020       __imp__GetCurrentProcessId@0 1000c020     kernel32:KERNEL32.dll
 0002:00000024       __imp__GetCurrentThreadId@0 1000c024     kernel32:KERNEL32.dll
 0002:00000028       __imp__GetSystemTimeAsFileTime@4 1000c028     kernel32:KERNEL32.dll
 0002:0000002c       __imp__DisableThreadLibraryCalls@4 1000c02c     kernel32:KERNEL32.dll
 0002:00000030       \177KERNEL32_NULL_THUNK_DATA 1000c030     kernel32:KERNEL32.dll
 0002:00000034       __imp___CxxThrowException@8 1000c034     vcruntime:VCRUNTIME140.dll
 0002:00000038       __imp____std_type_info_destroy_list 1000c038     vcruntime:VCRUNTIME140.dll
 0002:0000003c       __imp___except_handler4_common 1000c03c     vcruntime:VCRUNTIME140.dll
 0002:00000040       __imp____std_exception_destroy 1000c040     vcruntime:VCRUNTIME140.dll
 0002:00000044       __imp__memcmp              1000c044     vcruntime:VCRUNTIME140.dll
 0002:00000048       __imp__memcpy              1000c048     vcruntime:VCRUNTIME140.dll
 0002:0000004c       __imp__memset              1000c04c     vcruntime:VCRUNTIME140.dll
 0002:00000050       __imp__strchr              1000c050     vcruntime:VCRUNTIME140.dll
 0002:00000054       __imp____std_exception_copy 1000c054     vcruntime:VCRUNTIME140.dll
 0002:00000058       \177VCRUNTIME140_NULL_THUNK_DATA 1000c058     vcruntime:VCRUNTIME140.dll
 0002:0000005c       __imp__atoi                1000c05c     ucrt:api-ms-win-crt-convert-l1-1-0.dll
 0002:00000060       \177api-ms-win-crt-convert-l1-1-0_NULL_THUNK_DATA 1000c060     ucrt:api-ms-win-crt-convert-l1-1-0.dll
 0002:00000064       __imp__free                1000c064     ucrt:api-ms-win-crt-heap-l1-1-0.dll
 0002:00000068       __imp__realloc             1000c068     ucrt:api-ms-win-crt-heap-l1-1-0.dll
 0002:0000006c       __imp__calloc              1000c06c     ucrt:api-ms-win-crt-heap-l1-1-0.dll
 0002:00000070       __imp___callnewh           1000c070     ucrt:api-ms-win-crt-heap-l1-1-0.dll
 0002:00000074       __imp__malloc              1000c074     ucrt:api-ms-win-crt-heap-l1-1-0.dll
 0002:00000078       \177api-ms-win-crt-heap-l1-1-0_NULL_THUNK_DATA 1000c078     ucrt:api-ms-win-crt-heap-l1-1-0.dll
 0002:0000007c       __imp___initterm_e         1000c07c     ucrt:api-ms-win-crt-runtime-l1-1-0.dll
 0002:00000080       __imp___seh_filter_dll     1000c080     ucrt:api-ms-win-crt-runtime-l1-1-0.dll
 0002:00000084       __imp___configure_narrow_argv 1000c084     ucrt:api-ms-win-crt-runtime-l1-1-0.dll
 0002:00000088       __imp___cexit              1000c088     ucrt:api-ms-win-crt-runtime-l1-1-0.dll
 0002:0000008c       __imp___execute_onexit_table 1000c08c     ucrt:api-ms-win-crt-runtime-l1-1-0.dll
 0002:00000090       __imp___initterm           1000c090     ucrt:api-ms-win-crt-runtime-l1-1-0.dll
 0002:00000094       __imp__abort               1000c094     ucrt:api-ms-win-crt-runtime-l1-1-0.dll
 0002:00000098       __imp___initialize_onexit_table 1000c098     ucrt:api-ms-win-crt-runtime-l1-1-0.dll
 0002:0000009c       __imp___initialize_narrow_environment 1000c09c     ucrt:api-ms-win-crt-runtime-l1-1-0.dll
 0002:000000a0       \177api-ms-win-crt-runtime-l1-1-0_NULL_THUNK_DATA 1000c0a0     ucrt:api-ms-win-crt-runtime-l1-1-0.dll
 0002:000000a4       __imp____stdio_common_vsprintf 1000c0a4     ucrt:api-ms-win-crt-stdio-l1-1-0.dll
 0002:000000a8       __imp____stdio_common_vfprintf 1000c0a8     ucrt:api-ms-win-crt-stdio-l1-1-0.dll
 0002:000000ac       __imp__fopen               1000c0ac     ucrt:api-ms-win-crt-stdio-l1-1-0.dll
 0002:000000b0       __imp____acrt_iob_func     1000c0b0     ucrt:api-ms-win-crt-stdio-l1-1-0.dll
 0002:000000b4       \177api-ms-win-crt-stdio-l1-1-0_NULL_THUNK_DATA 1000c0b4     ucrt:api-ms-win-crt-stdio-l1-1-0.dll
 0002:000000b8       __imp__strcmp              1000c0b8     ucrt:api-ms-win-crt-string-l1-1-0.dll
 0002:000000bc       __imp__strlen              1000c0bc     ucrt:api-ms-win-crt-string-l1-1-0.dll
 0002:000000c0       __imp__strncat             1000c0c0     ucrt:api-ms-win-crt-string-l1-1-0.dll
 0002:000000c4       __imp__strcat              1000c0c4     ucrt:api-ms-win-crt-string-l1-1-0.dll
 0002:000000c8       \177api-ms-win-crt-string-l1-1-0_NULL_THUNK_DATA 1000c0c8     ucrt:api-ms-win-crt-string-l1-1-0.dll
 0002:000000cc       __imp___time64             1000c0cc     ucrt:api-ms-win-crt-time-l1-1-0.dll
 0002:000000d0       \177api-ms-win-crt-time-l1-1-0_NULL_THUNK_DATA 1000c0d0     ucrt:api-ms-win-crt-time-l1-1-0.dll
 0002:000000d4       __imp__qsort               1000c0d4     ucrt:api-ms-win-crt-utility-l1-1-0.dll
 0002:000000d8       \177api-ms-win-crt-utility-l1-1-0_NULL_THUNK_DATA 1000c0d8     ucrt:api-ms-win-crt-utility-l1-1-0.dll
 0002:000000dc       __imp__JNU_ThrowIOException@8 1000c0dc     java:java.dll
 0002:000000e0       \177java_NULL_THUNK_DATA   1000c0e0     java:java.dll
 0002:000000e4       __imp__JNI_GetCreatedJavaVMs@12 1000c0e4     jvm:jvm.dll
 0002:000000e8       \177jvm_NULL_THUNK_DATA    1000c0e8     jvm:jvm.dll
 0002:000000ec       ___guard_check_icall_fptr  1000c0ec     MSVCRT:guard_support.obj
 0002:000000f0       ___xc_a                    1000c0f0     MSVCRT:initializers.obj
 0002:000000f4       ___xc_z                    1000c0f4     MSVCRT:initializers.obj
 0002:000000f8       ___xi_a                    1000c0f8     MSVCRT:initializers.obj
 0002:000000fc       ___xi_z                    1000c0fc     MSVCRT:initializers.obj
 0002:00000100       ___xp_a                    1000c100     MSVCRT:initializers.obj
 0002:00000104       ___xp_z                    1000c104     MSVCRT:initializers.obj
 0002:00000108       ___xt_a                    1000c108     MSVCRT:initializers.obj
 0002:0000010c       ___xt_z                    1000c10c     MSVCRT:initializers.obj
 0002:00000ad0       ??_C@_0P@NFDCFGCL@cp_Utf8_prefix@ 1000cad0     bands.obj
 0002:00000ae0       ??_C@_0P@LOHPAGNO@cp_Utf8_suffix@ 1000cae0     bands.obj
 0002:00000af0       ??_C@_0O@IHLLKPBK@cp_Utf8_chars@ 1000caf0     bands.obj
 0002:00000b00       ??_C@_0BD@EOIEJGOP@cp_Utf8_big_suffix@ 1000cb00     bands.obj
 0002:00000b14       ??_C@_0BC@HDLINKIK@cp_Utf8_big_chars@ 1000cb14     bands.obj
 0002:00000b28       ??_C@_06IGKKGOEN@cp_Int@   1000cb28     bands.obj
 0002:00000b30       ??_C@_08OBBFNHHD@cp_Float@ 1000cb30     bands.obj
 0002:00000b3c       ??_C@_0L@HNFJMOEO@cp_Long_hi@ 1000cb3c     bands.obj
 0002:00000b48       ??_C@_0L@CMAKMBBE@cp_Long_lo@ 1000cb48     bands.obj
 0002:00000b54       ??_C@_0N@CPNNOOPC@cp_Double_hi@ 1000cb54     bands.obj
 0002:00000b64       ??_C@_0N@HOIOOBKI@cp_Double_lo@ 1000cb64     bands.obj
 0002:00000b74       ??_C@_09HFEHKGNE@cp_String@ 1000cb74     bands.obj
 0002:00000b80       ??_C@_08BOENACK@cp_Class@  1000cb80     bands.obj
 0002:00000b8c       ??_C@_0BC@FENMLAPO@cp_Signature_form@ 1000cb8c     bands.obj
 0002:00000ba0       ??_C@_0BF@MEOEAPGK@cp_Signature_classes@ 1000cba0     bands.obj
 0002:00000bb8       ??_C@_0O@JHMEINNJ@cp_Descr_name@ 1000cbb8     bands.obj
 0002:00000bc8       ??_C@_0O@DMMHENKJ@cp_Descr_type@ 1000cbc8     bands.obj
 0002:00000bd8       ??_C@_0P@EEAFDJFH@cp_Field_class@ 1000cbd8     bands.obj
 0002:00000be8       ??_C@_0O@FCFAPCDP@cp_Field_desc@ 1000cbe8     bands.obj
 0002:00000bf8       ??_C@_0BA@LDOOFFKI@cp_Method_class@ 1000cbf8     bands.obj
 0002:00000c08       ??_C@_0P@NLGLFAKL@cp_Method_desc@ 1000cc08     bands.obj
 0002:00000c18       ??_C@_0BB@IIGJKIIK@cp_Imethod_class@ 1000cc18     bands.obj
 0002:00000c2c       ??_C@_0BA@DCLGLKIL@cp_Imethod_desc@ 1000cc2c     bands.obj
 0002:00000c3c       ??_C@_0BI@NIJEEAN@cp_MethodHandle_refkind@ 1000cc3c     bands.obj
 0002:00000c54       ??_C@_0BH@NKNCKAEO@cp_MethodHandle_member@ 1000cc54     bands.obj
 0002:00000c6c       ??_C@_0O@NHPECHNH@cp_MethodType@ 1000cc6c     bands.obj
 0002:00000c7c       ??_C@_0BH@NPCIPIPL@cp_BootstrapMethod_ref@ 1000cc7c     bands.obj
 0002:00000c94       ??_C@_0BN@DJLEBMBH@cp_BootstrapMethod_arg_count@ 1000cc94     bands.obj
 0002:00000cb4       ??_C@_0BH@JNPGIEDO@cp_BootstrapMethod_arg@ 1000ccb4     bands.obj
 0002:00000ccc       ??_C@_0BG@CIPOMBAC@cp_InvokeDynamic_spec@ 1000cccc     bands.obj
 0002:00000ce4       ??_C@_0BG@IFFCPCPP@cp_InvokeDynamic_desc@ 1000cce4     bands.obj
 0002:00000cfc       ??_C@_0BI@KJJNKCHD@attr_definition_headers@ 1000ccfc     bands.obj
 0002:00000d14       ??_C@_0BF@EEAHHHEA@attr_definition_name@ 1000cd14     bands.obj
 0002:00000d2c       ??_C@_0BH@EKDDDJNL@attr_definition_layout@ 1000cd2c     bands.obj
 0002:00000d44       ??_C@_0O@HJMNFDHJ@ic_this_class@ 1000cd44     bands.obj
 0002:00000d54       ??_C@_08CKLAPDFF@ic_flags@ 1000cd54     bands.obj
 0002:00000d60       ??_C@_0P@MGLGIOLC@ic_outer_class@ 1000cd60     bands.obj
 0002:00000d70       ??_C@_07OPOCOJIH@ic_name@  1000cd70     bands.obj
 0002:00000d78       ??_C@_0L@GONOGKKN@class_this@ 1000cd78     bands.obj
 0002:00000d84       ??_C@_0M@FMPLOBH@class_super@ 1000cd84     bands.obj
 0002:00000d90       ??_C@_0BG@ELABOHHB@class_interface_count@ 1000cd90     bands.obj
 0002:00000da8       ??_C@_0BA@GDKGLIFF@class_interface@ 1000cda8     bands.obj
 0002:00000db8       ??_C@_0BC@GLACLOBG@class_field_count@ 1000cdb8     bands.obj
 0002:00000dcc       ??_C@_0BD@MFLGOFPO@class_method_count@ 1000cdcc     bands.obj
 0002:00000de0       ??_C@_0M@IINMAGFA@field_descr@ 1000cde0     bands.obj
 0002:00000dec       ??_C@_0P@LDBPJHCP@field_flags_hi@ 1000cdec     bands.obj
 0002:00000dfc       ??_C@_0P@OCEMJIHF@field_flags_lo@ 1000cdfc     bands.obj
 0002:00000e0c       ??_C@_0BB@GJGJJLKK@field_attr_count@ 1000ce0c     bands.obj
 0002:00000e20       ??_C@_0BD@LLAABMND@field_attr_indexes@ 1000ce20     bands.obj
 0002:00000e34       ??_C@_0BB@LHINHPHH@field_attr_calls@ 1000ce34     bands.obj
 0002:00000e48       ??_C@_0BH@NKCAAIDC@field_ConstantValue_KQ@ 1000ce48     bands.obj
 0002:00000e60       ??_C@_0BD@HMEKDNDB@field_Signature_RS@ 1000ce60     bands.obj
 0002:00000e74       ??_C@_0BF@KACJMLOM@field_metadata_bands@ 1000ce74     bands.obj
 0002:00000e8c       ??_C@_0BB@NIMLDFOB@field_attr_bands@ 1000ce8c     bands.obj
 0002:00000ea0       ??_C@_0N@GLCNNANE@method_descr@ 1000cea0     bands.obj
 0002:00000eb0       ??_C@_0BA@EIPLIEID@method_flags_hi@ 1000ceb0     bands.obj
 0002:00000ec0       ??_C@_0BA@BJKIILNJ@method_flags_lo@ 1000cec0     bands.obj
 0002:00000ed0       ??_C@_0BC@OPGFNCHF@method_attr_count@ 1000ced0     bands.obj
 0002:00000ee4       ??_C@_0BE@LCKALKDL@method_attr_indexes@ 1000cee4     bands.obj
 0002:00000ef8       ??_C@_0BC@DBIBDGKI@method_attr_calls@ 1000cef8     bands.obj
 0002:00000f0c       ??_C@_0BE@HAIBKECN@method_Exceptions_N@ 1000cf0c     bands.obj
 0002:00000f20       ??_C@_0BF@ILMHJLAD@method_Exceptions_RC@ 1000cf20     bands.obj
 0002:00000f38       ??_C@_0BE@HFOKJLNJ@method_Signature_RS@ 1000cf38     bands.obj
 0002:00000f4c       ??_C@_0BG@JDLLNHF@method_metadata_bands@ 1000cf4c     bands.obj
 0002:00000f64       ??_C@_0BL@MNBFAABE@method_MethodParameters_NB@ 1000cf64     bands.obj
 0002:00000f80       ??_C@_0CB@POGNKHAK@method_MethodParameters_name_RU@ 1000cf80     bands.obj
 0002:00000fa4       ??_C@_0CA@HDKLJONB@method_MethodParameters_flag_FH@ 1000cfa4     bands.obj
 0002:00000fc4       ??_C@_0BC@FOMHHMDO@method_attr_bands@ 1000cfc4     bands.obj
 0002:00000fd8       ??_C@_0P@DNMDIOJK@class_flags_hi@ 1000cfd8     bands.obj
 0002:00000fe8       ??_C@_0P@GMJAIBMA@class_flags_lo@ 1000cfe8     bands.obj
 0002:00000ff8       ??_C@_0BB@JELAOHEL@class_attr_count@ 1000cff8     bands.obj
 0002:0000100c       ??_C@_0BD@KFNGBOLA@class_attr_indexes@ 1000d00c     bands.obj
 0002:00001020       ??_C@_0BB@EKFEADJG@class_attr_calls@ 1000d020     bands.obj
 0002:00001034       ??_C@_0BF@MJNFEGEM@class_SourceFile_RUN@ 1000d034     bands.obj
 0002:0000104c       ??_C@_0BJ@CCGEELON@class_EnclosingMethod_RC@ 1000d04c     bands.obj
 0002:00001068       ??_C@_0BK@LFCMIOIA@class_EnclosingMethod_RDN@ 1000d068     bands.obj
 0002:00001084       ??_C@_0BD@GCJMDPFC@class_Signature_RS@ 1000d084     bands.obj
 0002:00001098       ??_C@_0BF@PHIMHC@class_metadata_bands@ 1000d098     bands.obj
 0002:000010b0       ??_C@_0BF@PGJMDHG@class_InnerClasses_N@ 1000d0b0     bands.obj
 0002:000010c8       ??_C@_0BG@HHABPLBI@class_InnerClasses_RC@ 1000d0c8     bands.obj
 0002:000010e0       ??_C@_0BF@MHLAEJHO@class_InnerClasses_F@ 1000d0e0     bands.obj
 0002:000010f8       ??_C@_0BN@FANFKEPF@class_InnerClasses_outer_RCN@ 1000d0f8     bands.obj
 0002:00001118       ??_C@_0BM@CHKHAMMI@class_InnerClasses_name_RUN@ 1000d118     bands.obj
 0002:00001134       ??_C@_0CA@LBNJCLO@class_ClassFile_version_minor_H@ 1000d134     bands.obj
 0002:00001154       ??_C@_0CA@KDGDJOMP@class_ClassFile_version_major_H@ 1000d154     bands.obj
 0002:00001174       ??_C@_0BB@CFBCEJAA@class_attr_bands@ 1000d174     bands.obj
 0002:00001188       ??_C@_0N@EJFJBMLJ@code_headers@ 1000d188     bands.obj
 0002:00001198       ??_C@_0P@DPBEANCA@code_max_stack@ 1000d198     bands.obj
 0002:000011a8       ??_C@_0BD@OBGMDNFJ@code_max_na_locals@ 1000d1a8     bands.obj
 0002:000011bc       ??_C@_0BD@OMMDBBC@code_handler_count@ 1000d1bc     bands.obj
 0002:000011d0       ??_C@_0BF@NAEEIJON@code_handler_start_P@ 1000d1d0     bands.obj
 0002:000011e8       ??_C@_0BE@GIJMHOG@code_handler_end_PO@ 1000d1e8     bands.obj
 0002:000011fc       ??_C@_0BG@GJGNOMGM@code_handler_catch_PO@ 1000d1fc     bands.obj
 0002:00001214       ??_C@_0BH@ECFPKFHF@code_handler_class_RCN@ 1000d214     bands.obj
 0002:0000122c       ??_C@_0O@PKFJGJJN@code_flags_hi@ 1000d22c     bands.obj
 0002:0000123c       ??_C@_0O@KLAKGGMH@code_flags_lo@ 1000d23c     bands.obj
 0002:0000124c       ??_C@_0BA@OFJPMBMN@code_attr_count@ 1000d24c     bands.obj
 0002:0000125c       ??_C@_0BC@BKACNFKP@code_attr_indexes@ 1000d25c     bands.obj
 0002:00001270       ??_C@_0BA@DLHLCFBA@code_attr_calls@ 1000d270     bands.obj
 0002:00001280       ??_C@_0BF@FNGGAIBD@code_StackMapTable_N@ 1000d280     bands.obj
 0002:00001298       ??_C@_0BL@IJLKAPMG@code_StackMapTable_frame_T@ 1000d298     bands.obj
 0002:000012b4       ??_C@_0BL@FLGOBHFL@code_StackMapTable_local_N@ 1000d2b4     bands.obj
 0002:000012d0       ??_C@_0BL@DBPDDGDK@code_StackMapTable_stack_N@ 1000d2d0     bands.obj
 0002:000012ec       ??_C@_0BK@HMGLLHPP@code_StackMapTable_offset@ 1000d2ec     bands.obj
 0002:00001308       ??_C@_0BF@ONELPCMI@code_StackMapTable_T@ 1000d308     bands.obj
 0002:00001320       ??_C@_0BG@EKILGBAE@code_StackMapTable_RC@ 1000d320     bands.obj
 0002:00001338       ??_C@_0BF@IJCHDHMM@code_StackMapTable_P@ 1000d338     bands.obj
 0002:00001350       ??_C@_0BH@EMJOIADC@code_LineNumberTable_N@ 1000d350     bands.obj
 0002:00001368       ??_C@_0BL@BODGMFAF@code_LineNumberTable_bci_P@ 1000d368     bands.obj
 0002:00001384       ??_C@_0BK@KMDHKKJP@code_LineNumberTable_line@ 1000d384     bands.obj
 0002:000013a0       ??_C@_0BK@EAEINMEG@code_LocalVariableTable_N@ 1000d3a0     bands.obj
 0002:000013bc       ??_C@_0BO@EBBJALKI@code_LocalVariableTable_bci_P@ 1000d3bc     bands.obj
 0002:000013dc       ??_C@_0BP@JIPNBFGM@code_LocalVariableTable_span_O@ 1000d3dc     bands.obj
 0002:000013fc       ??_C@_0CA@LBKLALLO@code_LocalVariableTable_name_RU@ 1000d3fc     bands.obj
 0002:0000141c       ??_C@_0CA@OBPDECDH@code_LocalVariableTable_type_RS@ 1000d41c     bands.obj
 0002:0000143c       ??_C@_0BN@BAELGOA@code_LocalVariableTable_slot@ 1000d43c     bands.obj
 0002:0000145c       ??_C@_0BO@HHCIFDPC@code_LocalVariableTypeTable_N@ 1000d45c     bands.obj
 0002:0000147c       ??_C@_0CC@OECAEAHA@code_LocalVariableTypeTable_bci@ 1000d47c     bands.obj
 0002:000014a0       ??_C@_0CD@BAFAHGMB@code_LocalVariableTypeTable_spa@ 1000d4a0     bands.obj
 0002:000014c4       ??_C@_0CE@BJEEHJII@code_LocalVariableTypeTable_nam@ 1000d4c4     bands.obj
 0002:000014e8       ??_C@_0CE@EJBMDAAB@code_LocalVariableTypeTable_typ@ 1000d4e8     bands.obj
 0002:0000150c       ??_C@_0CB@DCPKAFMH@code_LocalVariableTypeTable_slo@ 1000d50c     bands.obj
 0002:00001530       ??_C@_0BA@FEDNGPIG@code_attr_bands@ 1000d530     bands.obj
 0002:00001540       ??_C@_08ILNCKCLH@bc_codes@ 1000d540     bands.obj
 0002:0000154c       ??_C@_0O@NHDHOKJ@bc_case_count@ 1000d54c     bands.obj
 0002:0000155c       ??_C@_0O@IPODCEHE@bc_case_value@ 1000d55c     bands.obj
 0002:0000156c       ??_C@_07PBCCPPFP@bc_byte@  1000d56c     bands.obj
 0002:00001574       ??_C@_08LLANNIAP@bc_short@ 1000d574     bands.obj
 0002:00001580       ??_C@_08CNAAIOJJ@bc_local@ 1000d580     bands.obj
 0002:0000158c       ??_C@_08CNIFPPEB@bc_label@ 1000d58c     bands.obj
 0002:00001598       ??_C@_09LMIAJDCB@bc_intref@ 1000d598     bands.obj
 0002:000015a4       ??_C@_0M@GHNOKACA@bc_floatref@ 1000d5a4     bands.obj
 0002:000015b0       ??_C@_0L@FECALBEM@bc_longref@ 1000d5b0     bands.obj
 0002:000015bc       ??_C@_0N@BLIIPDNE@bc_doubleref@ 1000d5bc     bands.obj
 0002:000015cc       ??_C@_0N@MPKFBKGB@bc_stringref@ 1000d5cc     bands.obj
 0002:000015dc       ??_C@_0BE@JPNLPCGD@bc_loadablevalueref@ 1000d5dc     bands.obj
 0002:000015f0       ??_C@_0M@IBEIOBLC@bc_classref@ 1000d5f0     bands.obj
 0002:000015fc       ??_C@_0M@FHDAHFFG@bc_fieldref@ 1000d5fc     bands.obj
 0002:00001608       ??_C@_0N@KBJNFGEO@bc_methodref@ 1000d608     bands.obj
 0002:00001618       ??_C@_0O@BOILABNA@bc_imethodref@ 1000d618     bands.obj
 0002:00001628       ??_C@_0L@MEPMLOBJ@bc_indyref@ 1000d628     bands.obj
 0002:00001634       ??_C@_0N@CGLIFEKH@bc_thisfield@ 1000d634     bands.obj
 0002:00001644       ??_C@_0O@NMPFAKNK@bc_superfield@ 1000d644     bands.obj
 0002:00001654       ??_C@_0O@OCHHHCLJ@bc_thismethod@ 1000d654     bands.obj
 0002:00001664       ??_C@_0P@MMDJDCGG@bc_supermethod@ 1000d664     bands.obj
 0002:00001674       ??_C@_0L@IAPCGJHG@bc_initref@ 1000d674     bands.obj
 0002:00001680       ??_C@_09BGKIKDIC@bc_escref@ 1000d680     bands.obj
 0002:0000168c       ??_C@_0O@LHNEEOML@bc_escrefsize@ 1000d68c     bands.obj
 0002:0000169c       ??_C@_0L@HJKABJFB@bc_escsize@ 1000d69c     bands.obj
 0002:000016a8       ??_C@_0L@HOKHNNPG@bc_escbyte@ 1000d6a8     bands.obj
 0002:000016b4       ??_C@_09GOEDCGAO@file_name@ 1000d6b4     bands.obj
 0002:000016c0       ??_C@_0N@INICLDFG@file_size_hi@ 1000d6c0     bands.obj
 0002:000016d0       ??_C@_0N@NMNBLMAM@file_size_lo@ 1000d6d0     bands.obj
 0002:000016e0       ??_C@_0N@JMABFCDG@file_modtime@ 1000d6e0     bands.obj
 0002:000016f0       ??_C@_0N@OPKBLMJG@file_options@ 1000d6f0     bands.obj
 0002:00001700       ??_C@_08FPGGDHDD@no?5index@ 1000d700     bands.obj
 0002:0000170c       ??_C@_08CHILEFNK@null?5ref@ 1000d70c     bands.obj
 0002:00001718       ??_C@_07MLPLAPLE@bad?5ref@ 1000d718     bands.obj
 0002:00001720       ??_C@_0BC@CJBOIHCG@overflow?5detected@ 1000d720     bands.obj
 0002:00001734       ??_C@_0BJ@CALEAGEE@Native?5allocation?5failed@ 1000d734     bytes.obj
 0002:00001764       ??_C@_0BA@MMOCMGFH@bad?5value?5count@ 1000d764     coding.obj
 0002:00001774       ??_C@_0L@FLIJCFOD@bad?5coding@ 1000d774     coding.obj
 0002:00001780       ??_C@_0BE@IIPOPKNG@illegal?5arb?4?5coding@ 1000d780     coding.obj
 0002:00001794       ??_C@_0BF@OEPDPLDN@illegal?5run?5encoding@ 1000d794     coding.obj
 0002:000017ac       ??_C@_0BM@FJMGNNPG@illegal?5nested?5run?5encoding@ 1000d7ac     coding.obj
 0002:000017c8       ??_C@_0BF@JOAAKECG@illegal?5pop?5encoding@ 1000d7c8     coding.obj
 0002:000017e0       ??_C@_0BM@CDDFICON@illegal?5nested?5pop?5encoding@ 1000d7e0     coding.obj
 0002:000017fc       ??_C@_0BG@HLIJPJNL@pop?4L?5value?5too?5small@ 1000d7fc     coding.obj
 0002:00001814       ??_C@_0BH@OCEIAIEJ@pop?5token?5out?5of?5range@ 1000d814     coding.obj
 0002:0000182c       ??_C@_0CA@HBCNKKJO@bad?5meta?9coding?5for?5empty?5pop?1U@ 1000d82c     coding.obj
 0002:0000184c       ??_C@_0BA@DAENMACF@bad?5meta?9coding@ 1000d84c     coding.obj
 0002:0000185c       ??_C@_0P@DHEBFDOP@Internal?5error@ 1000d85c     jni.obj
 0002:0000186c       ??_C@_01LELAEKIP@J@        1000d86c     jni.obj
 0002:00001870       ??_C@_0M@ODCCEGO@unpackerPtr@ 1000d870     jni.obj
 0002:0000187c       ??_C@_0BK@MGOECGMC@cannot?5init?5class?5members@ 1000d87c     jni.obj
 0002:00001898       ??_C@_0BF@LHBAMMHC@?$CI?$CJLjava?1lang?1Object?$DL@ 1000d898     jni.obj
 0002:000018b0       ??_C@_0BA@HNJNGCPJ@currentInstance@ 1000d8b0     jni.obj
 0002:000018c0       ??_C@_0BK@KNKPMLAB@?$CILjava?1nio?1ByteBuffer?$DLJ?$CJJ@ 1000d8c0     jni.obj
 0002:000018dc       ??_C@_0M@OOANKPPH@readInputFn@ 1000d8dc     jni.obj
 0002:000018e8       ??_C@_03IGDHHNNC@?$CI?$CJJ@ 1000d8e8     jni.obj
 0002:000018ec       ??_C@_0P@BBAJIHLB@getUnpackerPtr@ 1000d8ec     jni.obj
 0002:0000192c       ??_C@_02DPKJAMEF@?$CFd@    1000d92c     unpack.obj
 0002:00001930       ??_C@_0BC@DHBHLEDC@bad?5utf8?5encoding@ 1000d930     unpack.obj
 0002:00001944       ??_C@_08MPEBFEBH@bad?5data@ 1000d944     unpack.obj
 0002:00001950       ??_C@_0BI@MCADJHPK@missing?5class?5reference@ 1000d950     unpack.obj
 0002:00001968       ??_C@_0BJ@DINDGABB@Internal?5buffer?5overflow@ 1000d968     unpack.obj
 0002:00001984       ??_C@_0BE@NBGJPKOJ@too?5much?5read?9ahead@ 1000d984     unpack.obj
 0002:00001998       ??_C@_0CB@MBENKFPE@EOF?5reading?5archive?5magic?5numbe@ 1000d998     unpack.obj
 0002:000019bc       ??_C@_0CF@INONBKGM@encountered?5a?5JAR?5header?5in?5unp@ 1000d9bc     unpack.obj
 0002:000019e8       ??_C@_0GN@MIAOKBBJ@?$EACorrupted?5pack?5file?3?5magic?1ver@ 1000d9e8     unpack.obj
 0002:00001a58       ??_C@_0DJ@EOFNCHGA@Format?5bits?5for?5Java?57?5must?5be?5@ 1000da58     unpack.obj
 0002:00001a94       ??_C@_0DH@PDJEDCEA@High?5archive?5option?5bits?5are?5re@ 1000da94     unpack.obj
 0002:00001acc       ??_C@_0BP@CKGMAJKP@EOF?5reading?5fixed?5input?5buffer@ 1000dacc     unpack.obj
 0002:00001aec       ??_C@_0BI@EDJMKDIH@impossible?5archive?5size@ 1000daec     unpack.obj
 0002:00001b04       ??_C@_0DE@HNNKIDEL@cannot?5allocate?5large?5input?5buf@ 1000db04     unpack.obj
 0002:00001b38       ??_C@_0BL@KOJPDLNM@EOF?5reading?5archive?5header@ 1000db38     unpack.obj
 0002:00001b54       ??_C@_0BJ@HODOOMDO@EOF?5reading?5band?5headers@ 1000db54     unpack.obj
 0002:00001b70       ??_C@_0DB@HCOAOCOI@archive?5too?5large?3?5?5constant?5po@ 1000db70     unpack.obj
 0002:00001ba4       ??_C@_0BA@BMKLBFBL@bad?5utf8?5suffix@ 1000dba4     unpack.obj
 0002:00001bb4       ??_C@_0BA@HHOGEFOO@bad?5utf8?5prefix@ 1000dbb4     unpack.obj
 0002:00001bc4       ??_C@_0BF@HNBIPEII@utf8?5prefix?5overflow@ 1000dbc4     unpack.obj
 0002:00001bdc       ??_C@_0BE@INMEHPDO@unexpected?5band?5?$CFs?6@ 1000dbdc     unpack.obj
 0002:00001bf0       ??_C@_0BKA@JMJPKLFN@01?$AASignature?$AADeprecated?$AARuntime@ 1000dbf0     unpack.obj
 0002:00001d90       ??_C@_0BK@NOGBJPAL@attribute?5index?5too?5large@ 1000dd90     unpack.obj
 0002:00001dac       ??_C@_0BK@OFNJKMED@redefined?5attribute?5index@ 1000ddac     unpack.obj
 0002:00001dc8       ??_C@_0BJ@OGDEGNBN@garbage?5at?5end?5of?5layout@ 1000ddc8     unpack.obj
 0002:00001de4       ??_C@_0BN@NJCEKHIO@garbage?5mixed?5with?5callables@ 1000dde4     unpack.obj
 0002:00001e04       ??_C@_0BD@BJONMNHI@bad?5call?5in?5layout@ 1000de04     unpack.obj
 0002:00001e18       ??_C@_0BD@EOHIHJFP@bad?5layout?5element@ 1000de18     unpack.obj
 0002:00001e2c       ??_C@_0BK@CHPLBKBJ@missing?5numeral?5in?5layout@ 1000de2c     unpack.obj
 0002:00001e46       ??_C@_00CNPNBAHC@@         1000de46     unpack.obj
 0002:00001e48       ??_C@_0BB@FJJKEHGJ@numeral?5overflow@ 1000de48     unpack.obj
 0002:00001e5c       ??_C@_0P@HDHNKEAB@bad?5union?5case@ 1000de5c     unpack.obj
 0002:00001e6c       ??_C@_0DD@PGOJPNFL@bad?5range?5in?5union?5case?5label?5?$CI@ 1000de6c     unpack.obj
 0002:00001ea0       ??_C@_0BO@JELFCPB@bad?5range?5in?5union?5case?5label@ 1000dea0     unpack.obj
 0002:00001ec0       ??_C@_0P@KBKJHJBF@bad?5case?5label@ 1000dec0     unpack.obj
 0002:00001ed0       ??_C@_0P@MNJPOPJO@bad?5call?5label@ 1000ded0     unpack.obj
 0002:00001ee0       ??_C@_0BF@ILAEDGAO@bad?5reference?5layout@ 1000dee0     unpack.obj
 0002:00001ef8       ??_C@_0BE@NGGDBALG@bad?5nested?5callable@ 1000def8     unpack.obj
 0002:00001f0c       ??_C@_0L@FLEMDFJG@bad?5layout@ 1000df0c     unpack.obj
 0002:00001f18       ??_C@_0JK@BMMFGJDP@?$FLNB?$FL?$CI1?$CJ?$FN?$FN?$FLNH?$FL?$CI1?$CJ?$FN?$FN?$FLRSHNH?$FLRUH?$CI1?$CJ@ 1000df18     unpack.obj
 0002:00001fb4       ??_C@_09MAEOCCFN@?$FLNB?$FL?$CI1?$CJ?$FN?$FN@ 1000dfb4     unpack.obj
 0002:00001fc0       ??_C@_0CC@PCCOCALL@?$FLNB?$FL?$CI1?$CJ?$FN?$FN?$FLNH?$FL?$CI1?$CJ?$FN?$FN?$FLRSHNH?$FLRUH?$CI1?$CJ@ 1000dfc0     unpack.obj
 0002:00001fe8       ??_C@_0BBL@GCIMMLOG@?$FLNH?$FL?$CI1?$CJ?$CI2?$CJ?$CI3?$CJ?$FN?$FN?$FLTB?$CI0?01?$CJ?$FLB?$FN?$CI16?$CJ?$FL@ 1000dfe8     unpack.obj
 0002:00002104       ??_C@_0BK@CIMGHPDJ@RuntimeVisibleAnnotations@ 1000e104     unpack.obj
 0002:00002120       ??_C@_0BM@BNNGFNMF@RuntimeInvisibleAnnotations@ 1000e120     unpack.obj
 0002:0000213c       ??_C@_0CD@ONLIBICP@RuntimeVisibleParameterAnnotati@ 1000e13c     unpack.obj
 0002:00002160       ??_C@_0CF@BFEAEHFK@RuntimeInvisibleParameterAnnota@ 1000e160     unpack.obj
 0002:00002188       ??_C@_0BC@DAGIEPHG@AnnotationDefault@ 1000e188     unpack.obj
 0002:0000219c       ??_C@_0BO@IJLELCEA@RuntimeVisibleTypeAnnotations@ 1000e19c     unpack.obj
 0002:000021bc       ??_C@_0CA@GCLMFPKD@RuntimeInvisibleTypeAnnotations@ 1000e1bc     unpack.obj
 0002:000021dc       ??_C@_0BG@FDJMCAOP@identical?5inner?5class@ 1000e1dc     unpack.obj
 0002:000021f4       ??_C@_0BN@GFADPNEE@undefined?5attribute?5flag?5bit@ 1000e1f4     unpack.obj
 0002:00002214       ??_C@_0BO@CMGKNLIA@attribute?5index?5out?5of?5bounds@ 1000e214     unpack.obj
 0002:00002234       ??_C@_0DH@OHIKFIJI@undefined?5StackMapTable?5attribu@ 1000e234     unpack.obj
 0002:0000226c       ??_C@_0CL@CLGKHLIF@layout_definition?5pointer?5must?5@ 1000e26c     unpack.obj
 0002:00002298       ??_C@_0CE@NENNCDNJ@putlayout?3?5unexpected?5NULL?5for?5@ 1000e298     unpack.obj
 0002:000022bc       ??_C@_0BB@HNCAJEIE@cp?5utf8?5overflow@ 1000e2bc     unpack.obj
 0002:000022d0       ??_C@_0BC@IJJDHGHN@cp?5class?5overflow@ 1000e2d0     unpack.obj
 0002:000022e4       ??_C@_0BE@DAFJFMML@unpack?4deflate?4hint@ 1000e2e4     unpack.obj
 0002:000022f8       ??_C@_0DC@KGJOKPLE@com?4sun?4java?4util?4jar?4pack?4unpa@ 1000e2f8     unpack.obj
 0002:0000232c       ??_C@_0CD@CEMFBAGC@com?4sun?4java?4util?4jar?4pack?4verb@ 1000e32c     unpack.obj
 0002:00002350       ??_C@_0DE@FNJPLIMN@com?4sun?4java?4util?4jar?4pack?4unpa@ 1000e350     unpack.obj
 0002:00002384       ??_C@_0CL@JFLJFCLE@com?4sun?4java?4util?4jar?4pack?4unpa@ 1000e384     unpack.obj
 0002:000023b0       ??_C@_04LKOEDJLC@keep@     1000e3b0     unpack.obj
 0002:000023b8       ??_C@_0CJ@LFNCLCEP@com?4sun?4java?4util?4jar?4pack?4verb@ 1000e3b8     unpack.obj
 0002:000023e4       ??_C@_03CGLHMDPP@now@      1000e3e4     unpack.obj
 0002:000023e8       ??_C@_01JOAMLHOP@?9@       1000e3e8     unpack.obj
 0002:000023ec       ??_C@_0BB@MNFIFPBF@bad?5KQ?5reference@ 1000e3ec     unpack.obj
 0002:00002400       ??_C@_0L@PDBBHOGB@bad?5bcimap@ 1000e400     unpack.obj
 0002:0000240c       ??_C@_0BM@GPDDEOEP@too?5many?5InnerClasses?5attrs@ 1000e40c     unpack.obj
 0002:00002428       ??_C@_05PBJILJE@?4java@    1000e428     unpack.obj
 0002:00002430       ??_C@_0BB@MICPNADP@bad?5layout?5index@ 1000e430     unpack.obj
 0002:00002444       ??_C@_0BE@BKLBLMJK@bad?5attribute?5index@ 1000e444     unpack.obj
 0002:00002458       ??_C@_0BN@CLDGGNCI@bad?5reference?5to?5inner?5class@ 1000e458     unpack.obj
 0002:00002478       ??_C@_0CC@IOEIADGN@archive?5header?5had?5incorrect?5si@ 1000e478     unpack.obj
 0002:0000249c       ??_C@_0BM@NDDMOHPH@class?5file?5size?5transmitted@ 1000e49c     unpack.obj
 0002:000024b8       ??_C@_06POIMOJKC@?4class@  1000e4b8     unpack.obj
 0002:000024c0       ??_C@_0BI@CDCINJGA@resource?5file?5too?5large@ 1000e4c0     unpack.obj
 0002:000024d8       ??_C@_02DPNLHKJD@a?$CL@    1000e4d8     unpack.obj
 0002:000024dc       ??_C@_0BK@NDLGHGBM@Can?5not?5open?5log?5file?5?$CFs?6@ 1000e4dc     unpack.obj
 0002:000024f8       ??_C@_0BI@CELHNJPG@error?5unpacking?5archive@ 1000e4f8     unpack.obj
 0002:00002510       __xmm@00000000000000ab00000001000000aa 1000e510     unpack.obj
 0002:00002520       __xmm@00000001000000a00000000700000096 1000e520     unpack.obj
 0002:00002530       ??_C@_0CE@HLJAOJEP@corrupt?5pack?5file?5or?5internal?5e@ 1000e530     utils.obj
 0002:00002554       ??_C@_0BF@JFFKOPFD@Error?3?5unpacker?3?5?$CFs?6@ 1000e554     utils.obj
 0002:0000256c       ??_C@_0CG@HFNCMKIN@Error?3?5unpacker?3?5no?5current?5ins@ 1000e56c     utils.obj
 0002:000025a0       __pDefaultRawDllMain       1000e5a0     MSVCRT:dll_dllmain.obj
 0002:000025a0       __pRawDllMain              1000e5a0     MSVCRT:dll_dllmain.obj
 0002:000025b0       ??_7exception@std@@6B@     1000e5b0     MSVCRT:throw_bad_alloc.obj
 0002:000025b8       ??_C@_0BC@EOODALEL@Unknown?5exception@ 1000e5b8     MSVCRT:throw_bad_alloc.obj
 0002:000025d0       ??_7bad_alloc@std@@6B@     1000e5d0     MSVCRT:throw_bad_alloc.obj
 0002:000025d8       ??_C@_0P@GHFPNOJB@bad?5allocation@ 1000e5d8     MSVCRT:throw_bad_alloc.obj
 0002:000025ec       ??_7bad_array_new_length@std@@6B@ 1000e5ec     MSVCRT:throw_bad_alloc.obj
 0002:000025f4       ??_C@_0BF@KINCDENJ@bad?5array?5new?5length@ 1000e5f4     MSVCRT:throw_bad_alloc.obj
 0002:00002610       ??_7type_info@@6B@         1000e610     MSVCRT:std_type_info_static.obj
 0002:00002690       __load_config_used         1000e690     MSVCRT:loadcfg.obj
 0002:00002730       ??_R4exception@std@@6B@    1000e730     MSVCRT:throw_bad_alloc.obj
 0002:00002744       ??_R3exception@std@@8      1000e744     MSVCRT:throw_bad_alloc.obj
 0002:00002754       ??_R2exception@std@@8      1000e754     MSVCRT:throw_bad_alloc.obj
 0002:0000275c       ??_R1A@?0A@EA@exception@std@@8 1000e75c     MSVCRT:throw_bad_alloc.obj
 0002:00002778       ??_R4bad_alloc@std@@6B@    1000e778     MSVCRT:throw_bad_alloc.obj
 0002:0000278c       ??_R3bad_alloc@std@@8      1000e78c     MSVCRT:throw_bad_alloc.obj
 0002:0000279c       ??_R2bad_alloc@std@@8      1000e79c     MSVCRT:throw_bad_alloc.obj
 0002:000027a8       ??_R1A@?0A@EA@bad_alloc@std@@8 1000e7a8     MSVCRT:throw_bad_alloc.obj
 0002:000027c4       ??_R4bad_array_new_length@std@@6B@ 1000e7c4     MSVCRT:throw_bad_alloc.obj
 0002:000027d8       ??_R3bad_array_new_length@std@@8 1000e7d8     MSVCRT:throw_bad_alloc.obj
 0002:000027e8       ??_R2bad_array_new_length@std@@8 1000e7e8     MSVCRT:throw_bad_alloc.obj
 0002:000027f8       ??_R1A@?0A@EA@bad_array_new_length@std@@8 1000e7f8     MSVCRT:throw_bad_alloc.obj
 0002:00002814       ??_R4type_info@@6B@        1000e814     MSVCRT:std_type_info_static.obj
 0002:00002828       ??_R3type_info@@8          1000e828     MSVCRT:std_type_info_static.obj
 0002:00002838       ??_R2type_info@@8          1000e838     MSVCRT:std_type_info_static.obj
 0002:00002840       ??_R1A@?0A@EA@type_info@@8 1000e840     MSVCRT:std_type_info_static.obj
 0002:00002860       ___safe_se_handler_table   1000e860     <linker-defined>
 0002:00002b0c       ___rtc_iaa                 1000eb0c     MSVCRT:initsect.obj
 0002:00002b10       ___rtc_izz                 1000eb10     MSVCRT:initsect.obj
 0002:00002b14       ___rtc_taa                 1000eb14     MSVCRT:initsect.obj
 0002:00002b18       ___rtc_tzz                 1000eb18     MSVCRT:initsect.obj
 0002:00002b7c       __TI2?AVbad_alloc@std@@    1000eb7c     MSVCRT:throw_bad_alloc.obj
 0002:00002b8c       __CTA2?AVbad_alloc@std@@   1000eb8c     MSVCRT:throw_bad_alloc.obj
 0002:00002b98       __CT??_R0?AVbad_alloc@std@@@8??0bad_alloc@std@@QAE@ABV01@@Z12 1000eb98     MSVCRT:throw_bad_alloc.obj
 0002:00002bb4       __CT??_R0?AVexception@std@@@8??0exception@std@@QAE@ABV01@@Z12 1000ebb4     MSVCRT:throw_bad_alloc.obj
 0002:00002bd0       __TI3?AVbad_array_new_length@std@@ 1000ebd0     MSVCRT:throw_bad_alloc.obj
 0002:00002be0       __CTA3?AVbad_array_new_length@std@@ 1000ebe0     MSVCRT:throw_bad_alloc.obj
 0002:00002bf0       __CT??_R0?AVbad_array_new_length@std@@@8??0bad_array_new_length@std@@QAE@ABV01@@Z12 1000ebf0     MSVCRT:throw_bad_alloc.obj
 0002:00002e44       __IMPORT_DESCRIPTOR_jvm    1000ee44     jvm:jvm.dll
 0002:00002e58       __IMPORT_DESCRIPTOR_java   1000ee58     java:java.dll
 0002:00002e6c       __IMPORT_DESCRIPTOR_KERNEL32 1000ee6c     kernel32:KERNEL32.dll
 0002:00002e80       __IMPORT_DESCRIPTOR_VCRUNTIME140 1000ee80     vcruntime:VCRUNTIME140.dll
 0002:00002e94       __IMPORT_DESCRIPTOR_api-ms-win-crt-heap-l1-1-0 1000ee94     ucrt:api-ms-win-crt-heap-l1-1-0.dll
 0002:00002ea8       __IMPORT_DESCRIPTOR_api-ms-win-crt-stdio-l1-1-0 1000eea8     ucrt:api-ms-win-crt-stdio-l1-1-0.dll
 0002:00002ebc       __IMPORT_DESCRIPTOR_api-ms-win-crt-string-l1-1-0 1000eebc     ucrt:api-ms-win-crt-string-l1-1-0.dll
 0002:00002ed0       __IMPORT_DESCRIPTOR_api-ms-win-crt-utility-l1-1-0 1000eed0     ucrt:api-ms-win-crt-utility-l1-1-0.dll
 0002:00002ee4       __IMPORT_DESCRIPTOR_api-ms-win-crt-convert-l1-1-0 1000eee4     ucrt:api-ms-win-crt-convert-l1-1-0.dll
 0002:00002ef8       __IMPORT_DESCRIPTOR_api-ms-win-crt-time-l1-1-0 1000eef8     ucrt:api-ms-win-crt-time-l1-1-0.dll
 0002:00002f0c       __IMPORT_DESCRIPTOR_api-ms-win-crt-runtime-l1-1-0 1000ef0c     ucrt:api-ms-win-crt-runtime-l1-1-0.dll
 0002:00002f20       __NULL_IMPORT_DESCRIPTOR   1000ef20     jvm:jvm.dll
 0003:00000000       ?basic_codings@@3PAUcoding@@A 10010000     coding.obj
 0003:00000af8       ___security_cookie_complement 10010af8     MSVCRT:gs_cookie.obj
 0003:00000afc       ___security_cookie         10010afc     MSVCRT:gs_cookie.obj
 0003:00000b00       ___scrt_native_dllmain_reason 10010b00     MSVCRT:utility.obj
 0003:00000b10       ___isa_enabled             10010b10     MSVCRT:cpu_disp.obj
 0003:00000b14       ___scrt_ucrt_dll_is_in_use 10010b14     MSVCRT:ucrt_stubs.obj
 0003:00000b18       ??_R0?AVbad_alloc@std@@@8  10010b18     MSVCRT:throw_bad_alloc.obj
 0003:00000b34       ??_R0?AVexception@std@@@8  10010b34     MSVCRT:throw_bad_alloc.obj
 0003:00000b50       ??_R0?AVbad_array_new_length@std@@@8 10010b50     MSVCRT:throw_bad_alloc.obj
 0003:00000b78       ??_R0?AVtype_info@@@8      10010b78     MSVCRT:std_type_info_static.obj
 0003:00000fa8       ?_OptionsStorage@?1??__local_stdio_printf_options@@9@4_KA 10010fa8     unpack.obj
 0003:000012d8       ?__type_info_root_node@@3U__type_info_node@@A 100112d8     MSVCRT:tncleanup.obj
 0003:000012e0       ?_OptionsStorage@?1??__local_stdio_scanf_options@@9@4_KA 100112e0     MSVCRT:default_local_stdio_options.obj
 0003:000012e8       ___scrt_current_native_startup_state 100112e8     MSVCRT:utility.obj
 0003:000012ec       ___scrt_native_startup_lock 100112ec     MSVCRT:utility.obj
 0003:0000130c       ___scrt_debugger_hook_flag 1001130c     MSVCRT:utility_desktop.obj
 0003:00001310       ___isa_available           10011310     MSVCRT:cpu_disp.obj
 0003:00001314       ___favor                   10011314     MSVCRT:cpu_disp.obj
 0003:00001318       ___dyn_tls_init_callback   10011318     <common>

 entry point at        0001:00009f5f

 Static symbols

 0000:fffec000       .debug$S                   10000000     kernel32:KERNEL32.dll
 0000:fffec000       .debug$S                   10000000     kernel32:KERNEL32.dll
 0000:fffec000       .debug$S                   10000000     kernel32:KERNEL32.dll
 0000:fffec000       .debug$S                   10000000     kernel32:KERNEL32.dll
 0000:fffec000       .debug$S                   10000000     kernel32:KERNEL32.dll
 0000:fffec000       .debug$S                   10000000     kernel32:KERNEL32.dll
 0000:fffec000       .debug$S                   10000000     kernel32:KERNEL32.dll
 0000:fffec000       .debug$S                   10000000     kernel32:KERNEL32.dll
 0000:fffec000       .debug$S                   10000000     kernel32:KERNEL32.dll
 0000:fffec000       .debug$S                   10000000     kernel32:KERNEL32.dll
 0000:fffec000       .debug$S                   10000000     kernel32:KERNEL32.dll
 0000:fffec000       .debug$S                   10000000     kernel32:KERNEL32.dll
 0000:fffec000       .debug$S                   10000000     unpack.exp
 0000:fffec000       .debug$S                   10000000     kernel32:KERNEL32.dll
 0002:ffff4000       .idata$6                   10000000     ucrt:api-ms-win-crt-filesystem-l1-1-0.dll
 0000:fffec000       .debug$S                   10000000     kernel32:KERNEL32.dll
 0000:fffec000       .debug$S                   10000000     java:java.dll
 0000:fffec000       .debug$S                   10000000     vcruntime:VCRUNTIME140.dll
 0000:fffec000       .debug$S                   10000000     vcruntime:VCRUNTIME140.dll
 0000:fffec000       .debug$S                   10000000     vcruntime:VCRUNTIME140.dll
 0000:fffec000       .debug$S                   10000000     vcruntime:VCRUNTIME140.dll
 0000:fffec000       .debug$S                   10000000     vcruntime:VCRUNTIME140.dll
 0000:fffec000       .debug$S                   10000000     ucrt:api-ms-win-crt-filesystem-l1-1-0.dll
 0000:fffec000       .debug$S                   10000000     ucrt:api-ms-win-crt-runtime-l1-1-0.dll
 0000:fffec000       .debug$S                   10000000     ucrt:api-ms-win-crt-runtime-l1-1-0.dll
 0000:fffec000       .debug$S                   10000000     ucrt:api-ms-win-crt-runtime-l1-1-0.dll
 0000:fffec000       .debug$S                   10000000     ucrt:api-ms-win-crt-runtime-l1-1-0.dll
 0000:fffec000       .debug$S                   10000000     ucrt:api-ms-win-crt-runtime-l1-1-0.dll
 0000:fffec000       .debug$S                   10000000     ucrt:api-ms-win-crt-runtime-l1-1-0.dll
 0000:fffec000       .debug$S                   10000000     ucrt:api-ms-win-crt-runtime-l1-1-0.dll
 0000:fffec000       .debug$S                   10000000     ucrt:api-ms-win-crt-runtime-l1-1-0.dll
 0000:fffec000       .debug$S                   10000000     ucrt:api-ms-win-crt-runtime-l1-1-0.dll
 0000:fffec000       .debug$S                   10000000     ucrt:api-ms-win-crt-runtime-l1-1-0.dll
 0000:fffec000       .debug$S                   10000000     ucrt:api-ms-win-crt-runtime-l1-1-0.dll
 0000:fffec000       .debug$S                   10000000     ucrt:api-ms-win-crt-runtime-l1-1-0.dll
 0000:fffec000       .debug$S                   10000000     ucrt:api-ms-win-crt-heap-l1-1-0.dll
 0000:fffec000       .debug$S                   10000000     ucrt:api-ms-win-crt-heap-l1-1-0.dll
 0000:fffec000       .debug$S                   10000000     ucrt:api-ms-win-crt-runtime-l1-1-0.dll
 0000:fffec000       .debug$S                   10000000     ucrt:api-ms-win-crt-time-l1-1-0.dll
 0000:fffec000       .debug$S                   10000000     ucrt:api-ms-win-crt-runtime-l1-1-0.dll
 0000:fffec000       .debug$S                   10000000     ucrt:api-ms-win-crt-stdio-l1-1-0.dll
 0000:fffec000       .debug$S                   10000000     ucrt:api-ms-win-crt-string-l1-1-0.dll
 0000:fffec000       .debug$S                   10000000     ucrt:api-ms-win-crt-runtime-l1-1-0.dll
 0000:fffec000       .debug$S                   10000000     ucrt:api-ms-win-crt-heap-l1-1-0.dll
 0000:fffec000       .debug$S                   10000000     ucrt:api-ms-win-crt-time-l1-1-0.dll
 0000:fffec000       .debug$S                   10000000     ucrt:api-ms-win-crt-convert-l1-1-0.dll
 0000:fffec000       .debug$S                   10000000     ucrt:api-ms-win-crt-utility-l1-1-0.dll
 0000:fffec000       .debug$S                   10000000     ucrt:api-ms-win-crt-string-l1-1-0.dll
 0000:fffec000       .debug$S                   10000000     ucrt:api-ms-win-crt-string-l1-1-0.dll
 0000:fffec000       .debug$S                   10000000     ucrt:api-ms-win-crt-string-l1-1-0.dll
 0000:fffec000       .debug$S                   10000000     ucrt:api-ms-win-crt-string-l1-1-0.dll
 0000:fffec000       .debug$S                   10000000     ucrt:api-ms-win-crt-stdio-l1-1-0.dll
 0000:fffec000       .debug$S                   10000000     ucrt:api-ms-win-crt-stdio-l1-1-0.dll
 0000:fffec000       .debug$S                   10000000     ucrt:api-ms-win-crt-stdio-l1-1-0.dll
 0000:fffec000       .debug$S                   10000000     ucrt:api-ms-win-crt-stdio-l1-1-0.dll
 0000:fffec000       .debug$S                   10000000     ucrt:api-ms-win-crt-stdio-l1-1-0.dll
 0000:fffec000       .debug$S                   10000000     ucrt:api-ms-win-crt-stdio-l1-1-0.dll
 0000:fffec000       .debug$S                   10000000     ucrt:api-ms-win-crt-heap-l1-1-0.dll
 0000:fffec000       .debug$S                   10000000     ucrt:api-ms-win-crt-heap-l1-1-0.dll
 0000:fffec000       .debug$S                   10000000     jvm:jvm.dll
 0000:fffec000       .debug$S                   10000000     vcruntime:VCRUNTIME140.dll
 0000:fffec000       .debug$S                   10000000     vcruntime:VCRUNTIME140.dll
 0000:fffec000       .debug$S                   10000000     vcruntime:VCRUNTIME140.dll
 0000:fffec000       .debug$S                   10000000     vcruntime:VCRUNTIME140.dll
 0000:fffec000       .debug$S                   10000000     vcruntime:VCRUNTIME140.dll
 0000:fffec000       .debug$S                   10000000     vcruntime:VCRUNTIME140.dll
 0001:0000075f       ?decode_sign@@YAHHI@Z      1000175f f   coding.obj
 0001:00000853       ?getDeltaValue@@YAHPAUvalue_stream@@I_N@Z 10001853 f   coding.obj
 0001:00000a87       $LN57                      10001a87     coding.obj
 0001:00000ac7       ?getPopValue@@YAHPAUvalue_stream@@I@Z 10001ac7 f   coding.obj
 0001:000016f1       ?free_unpacker@@YAXPAUJNIEnv_@@PAV_jobject@@PAUunpacker@@@Z 100026f1 f   jni.obj
 0001:00001738       ?get_unpacker@@YAPAUunpacker@@PAUJNIEnv_@@PAV_jobject@@_N@Z 10002738 f   jni.obj
 0001:000017c9       ?get_unpacker@@YAPAUunpacker@@XZ 100027c9 f   jni.obj
 0001:00001854       ?read_input_via_jni@@YA_JPAUunpacker@@PAX_J2@Z 10002854 f   jni.obj
 0001:000020d2       ?compare_Utf8_chars@@YAHAAUbytes@@0@Z 100030d2 f   unpack.obj
 0001:000035ac       ?isDigitString@@YA_NAAUbytes@@HH@Z 100045ac f   unpack.obj
 0001:0000360b       ?isLoadableValue@@YA_NH@Z  1000460b f   unpack.obj
 0001:00003673       ?is_branch_op@@YA_NH@Z     10004673 f   unpack.obj
 0001:00003693       ?is_local_slot_op@@YA_NH@Z 10004693 f   unpack.obj
 0001:000036bd       ?lastIndexOf@@YAHHHAAUbytes@@H@Z 100046bd f   unpack.obj
 0001:000062a7       $LN67                      100072a7     unpack.obj
 0001:00007675       $LN21                      10008675     unpack.obj
 0001:00007ab2       ?store_Utf8_char@@YAPACPACG@Z 10008ab2 f   unpack.obj
 0001:00009089       $LN51                      1000a089     unpack.obj
 0001:000090a5       $LN48                      1000a0a5     unpack.obj
 0001:00009ba0       $$000000                   1000aba0     MSVCRT:llmul.obj
 0001:00009c20       $$000000                   1000ac20     MSVCRT:ullshr.obj
 0001:00009c3f       ?dllmain_crt_dispatch@@YGHQAUHINSTANCE__@@KQAX@Z 1000ac3f f   MSVCRT:dll_dllmain.obj
 0001:00009c92       ?dllmain_crt_process_attach@@YAHQAUHINSTANCE__@@QAX@Z 1000ac92 f   MSVCRT:dll_dllmain.obj
 0001:00009d9c       ?dllmain_crt_process_detach@@YAH_N@Z 1000ad9c f   MSVCRT:dll_dllmain.obj
 0001:00009e2e       ?dllmain_dispatch@@YAHQAUHINSTANCE__@@KQAX@Z 1000ae2e f   MSVCRT:dll_dllmain.obj
 0001:00009f34       ?dllmain_raw@@YGHQAUHINSTANCE__@@KQAX@Z 1000af34 f   MSVCRT:dll_dllmain.obj
 0001:0000a1c1       ___get_entropy             1000b1c1 f   MSVCRT:gs_support.obj
 0001:0000a2b6       ?find_pe_section@@YAPAU_IMAGE_SECTION_HEADER@@QAEI@Z 1000b2b6 f   MSVCRT:utility.obj
 0001:0000a730       $$000000                   1000b730     MSVCRT:sehprolg4.obj
 0002:00000110       ?all_band_inits@@3QBUband_init@@B 1000c110     bands.obj
 0002:00001750       ?ERB@@3QBDB                1000d750     coding.obj
 0002:000018fc       ?TAGS_IN_ORDER@@3QBCB      1000d8fc     unpack.obj
 0002:0000190c       ?TAG_ORDER@@3QBCB          1000d90c     unpack.obj
 0002:00001920       ?str_tf@@3QBDB             1000d920     unpack.obj
 0002:00002594       ?jarmagic@@3QBGB           1000e594     zip.obj
 0002:00002598       ?marker_comment@@3QBDB     1000e598     zip.obj
 0002:000025a4       _GS_ExceptionPointers      1000e5a4     MSVCRT:gs_report.obj
 0002:00002b20       __sehtable$?dllmain_crt_process_attach@@YAHQAUHINSTANCE__@@QAX@Z 1000eb20     MSVCRT:dll_dllmain.obj
 0002:00002b40       __sehtable$?dllmain_crt_process_detach@@YAH_N@Z 1000eb40     MSVCRT:dll_dllmain.obj
 0002:00002b60       __sehtable$?dllmain_dispatch@@YAHQAUHINSTANCE__@@KQAX@Z 1000eb60     MSVCRT:dll_dllmain.obj
 0002:00002c10       __sehtable$___scrt_is_nonwritable_in_current_image 1000ec10     MSVCRT:utility.obj
 0002:00002c30       .edata                     1000ec30     unpack.exp
 0002:00002c58       rgpv                       1000ec58     unpack.exp
 0002:00002c74       rgszName                   1000ec74     unpack.exp
 0002:00002c90       rgwOrd                     1000ec90     unpack.exp
 0002:00002c9e       szName                     1000ec9e     unpack.exp
 0002:00002ca9       $N00001                    1000eca9     unpack.exp
 0002:00002ce0       $N00002                    1000ece0     unpack.exp
 0002:00002d1d       $N00003                    1000ed1d     unpack.exp
 0002:00002d58       $N00004                    1000ed58     unpack.exp
 0002:00002d97       $N00005                    1000ed97     unpack.exp
 0002:00002dcf       $N00006                    1000edcf     unpack.exp
 0002:00002e0a       $N00007                    1000ee0a     unpack.exp
 0002:00003038       .idata$6                   1000f038     jvm:jvm.dll
 0002:0000305a       .idata$6                   1000f05a     java:java.dll
 0002:00003188       .idata$6                   1000f188     kernel32:KERNEL32.dll
 0002:00003240       .idata$6                   1000f240     vcruntime:VCRUNTIME140.dll
 0002:000033c2       .idata$6                   1000f3c2     ucrt:api-ms-win-crt-heap-l1-1-0.dll
 0002:000033e2       .idata$6                   1000f3e2     ucrt:api-ms-win-crt-stdio-l1-1-0.dll
 0002:00003402       .idata$6                   1000f402     ucrt:api-ms-win-crt-string-l1-1-0.dll
 0002:00003424       .idata$6                   1000f424     ucrt:api-ms-win-crt-utility-l1-1-0.dll
 0002:00003446       .idata$6                   1000f446     ucrt:api-ms-win-crt-convert-l1-1-0.dll
 0002:00003468       .idata$6                   1000f468     ucrt:api-ms-win-crt-time-l1-1-0.dll
 0002:00003488       .idata$6                   1000f488     ucrt:api-ms-win-crt-runtime-l1-1-0.dll
 0003:00000b90       ?dummy@@3PACA              10010b90     bytes.obj
 0003:00000f90       ?no_meta@@3PAPBCA          10010f90     coding.obj
 0003:00000f94       ?unpackerPtrFID@@3PAU_jfieldID@@A 10010f94     jni.obj
 0003:00000f98       ?currentInstMID@@3PAU_jmethodID@@A 10010f98     jni.obj
 0003:00000f9c       ?readInputMID@@3PAU_jmethodID@@A 10010f9c     jni.obj
 0003:00000fa0       ?NIclazz@@3PAV_jclass@@A   10010fa0     jni.obj
 0003:00000fa4       ?getUnpackerPtrMID@@3PAU_jmethodID@@A 10010fa4     jni.obj
 0003:00000fb0       ?no_bands@@3PAPAUband@@A   10010fb0     unpack.obj
 0003:00000fb4       ?__proc_attached@@3HA      10010fb4     MSVCRT:dll_dllmain.obj
 0003:00000fb8       _GS_ExceptionRecord        10010fb8     MSVCRT:gs_report.obj
 0003:00001008       _GS_ContextRecord          10011008     MSVCRT:gs_report.obj
 0003:000012f0       ?is_initialized_as_dll@@3_NA 100112f0     MSVCRT:utility.obj
 0003:000012f1       ?module_local_atexit_table_initialized@@3_NA 100112f1     MSVCRT:utility.obj
 0003:000012f4       ?module_local_atexit_table@@3U_onexit_table_t@@A 100112f4     MSVCRT:utility.obj
 0003:00001300       ?module_local_at_quick_exit_table@@3U_onexit_table_t@@A 10011300     MSVCRT:utility.obj
 0004:00000060       $R000000                   10012060     unpack.dll.res
